:100000001DC2000038C2000036C2000034C2000029
:1000100032C2000030C200002EC200002CC200001C
:100020002AC2000028C200000C94B72E0C949C2F0A
:100030000C94BD0F20C200001EC200001CC20000B4
:100040001AC2000018C2000016C2000014C200004C
:1000500012C200000C94932E0EC200000CC20000CD
:100060000AC2000008C2000006C2000004C200006C
:1000700002C2000000C20000FEC10000FCC100007E
:10008000FAC10000F8C10000F6C10000F4C1000090
:10009000F2C10000F0C10000EEC10000ECC10000A0
:1000A000EAC10000E8C10000E6C100000501090244
:1000B000A10185020901A1000509190129081500FE
:1000C0002501950875018102050109300931158165
:1000D000257F95027508810609381581257F9501D0
:1000E00075088106050C0A38021581257F95017572
:1000F000088106C0C005010980A101850319012AF4
:10010000B700150126B700950175108100C0050CD8
:100110000901A101850419012AA002150126A002E6
:10012000950175108100C00660FF0961A101096297
:10013000150026FF00952075088102096315002629
:10014000FF00952075089102C005010906A101056F
:100150000719E029E7150025019508750181029529
:1001600001750881010507190029FF150026FF0008
:100170009506750881000508190129051500250156
:10018000950575019102950175039101C00000006C
:10019000000000000000000000000000000000005F
:1001A000000000000000000000000000000000004F
:1001B000007E0F00D4FFFFFFC700000078000000A2
:1001C00000000000002A2B280000000000000000B2
:1001D000000000000000000029000000002C1E3478
:1001E00020212224342627252E362D3738271E1F7E
:1001F000202122232425263333362E37381F0405A9
:10020000060708090A0B0C0D0E0F10111213141516
:10021000161718191A1B1C1D2F3130232D350405F4
:10022000060708090A0B0C0D0E0F101112131415F6
:10023000161718191A1B1C1D2F3130354C09025B7B
:1002400000030100A03209040000010301010009BC
:100250002111010001224400070581030800010962
:100260000401000203000000092111010001222203
:100270000007058203200001070503032000010990
:100280000402000103000000092111010001227B8A
:10029000000705840320000112010002000000088D
:1002A000435042540100010203011C03760069001F
:1002B00061006C003A0066003600340063003200D2
:1002C0006200330063000000240343006C006100FF
:1002D0007300730069006300200054007200610025
:1002E00063006B00620061006C006C0000000E0394
:1002F00050006C006F006F00700079000000040374
:100300000904D100D300D200D400D500FD377A58BB
:100310005A000004E6D6B44602002101160000008F
:10032000742FE5A3E0018800EF5D003D8889C65485
:1003300036C3174FE4E468771740EC062B597590E5
:10034000EA1B9E88D5853C2B2D4649B919FCF467DC
:10035000F3A7C15AE35727ECA65FCF01EFA012F332
:1003600075408571C8B6B71AD95082EFCEEC022C11
:100370004BF169D1ADF2D35939B7ECCF0C68A31A60
:10038000230109F1C2D35B7E87CC6DA17641DF18D2
:1003900080A47EAE025DCA7A3D0428A38325519ACB
:1003A000FF214AB537E83ED7103AB24F82E5DD9BD0
:1003B000990185D12E28DDC1DDFF435BE43FA12CEF
:1003C000C43E82271EE55CF80163364014C837E45A
:1003D000C4547DD3F980451BCBCF840E89562F02A0
:1003E000603F17246BEC672929A3A6AF9B076E908B
:1003F000BCE811B79AF314DFF8395779205B05D6BA
:10040000014BF2B2346B9D15EDBB99D53498EECB10
:100410002A711B840FF78AE71C00000079A72A4283
:100420008977A32D00018B02890300004E24F55F1C
:10043000B1C467FB020000000004595A11241FBE1A
:10044000CFEFDAE0DEBFCDBF11E0A0E0B1E0EAED32
:10045000F8E602C005900D92A43BB107D9F725E05C
:10046000A4EBB1E001C01D92A53DB207E1F70E94E7
:1004700011260C94F133C4CDA4E0B0E0E2E4F2E044
:100480000C947C312C01FB013A0129833A830B83C4
:100490001C831701960185017401898C9A8C8081D7
:1004A00091814816590614F451824082D301CD90AF
:1004B000DC901197C414D5041CF44D925C92620137
:1004C000A080B180C6018A199B098A309105ECF1A0
:1004D00063E070E00E94C7316A0D7B1D4616570627
:1004E0000CF07BC0AB81BC818C91811509F470C08C
:1004F000D7018D919C91DC01AA0FBB1FA20FB31FE6
:10050000CD92DC92D7018D919C9111978E319105FE
:100510000CF057C001968D939C9340815181D3017B
:100520008D919C91841B950B97FD019695958795D0
:10053000840F951F91838083D3018D939C93A98110
:10054000BA811C92AB81BC811C92AB8DBC8D8C910D
:10055000811509F466C0D901225C3F4F80E090E02C
:100560004D915D91840F951F2A173B07C9F76FE1E5
:1005700070E00E94C7319B01D4018C91811509F470
:1005800069C0F101A101425C5F4F80E090E06191A0
:100590007191860F971F4E175F07C9F76FE170E0E3
:1005A0000E94C731FB01C9018E1B9F0B63E070E005
:1005B0000E94C731CB018E0F9F1F2496E2E10C945D
:1005C00098311D921C9281E0AB8DBC8D8C93A5CF90
:1005D00081E0A981BA818C93B8CF641575050CF0C0
:1005E000B4CFA981BA818C918115B9F0D8018D91D0
:1005F0009C91DC01AA0FBB1FA20DB31DAD92BC9252
:10060000D8018D919C9111978E3191050CF482CF78
:100610001D921C9281E0D401D9CF81E0AB81BC81D5
:10062000DACFD7016D917C91D90120E030E080E0F4
:1006300090E06115710551F4D3012D913C919CCF4F
:100640004D915D91840F951F2F5F3F4F2617370700
:10065000BCF38FCFD8016D917C916115710581F04C
:10066000F10140E050E080E090E0461757070CF0C1
:1006700097CFA191B1918A0F9B1F4F5F5F4FF5CF2D
:100680000190F081E02D8FCF9C019A9581159F41BB
:1006900018F5F32FF270EE27832F8170732F74708B
:1006A0006627532F5870442734FF0CC08295807FF3
:1006B000EF2B09F08062672B09F08064452B69F00D
:1006C00080680895EF2B09F08260672B09F0846041
:1006D000452B19F08860089580E00895CF93DF934B
:1006E000EB01D2DFFE010995DF91CF910895809350
:1006F000CB0508958093CC05089521E030E001C03A
:10070000220F8A95EAF78091CC05822BF3CF21E066
:1007100030E0A90102C0440F551F8A95E2F7CA01D3
:1007200080959091CC058923E5CF911121C085302A
:10073000F8F491E001C0990F8A95EAF7892FE8EE65
:10074000F3E040E050E070E09191DF019B01042E66
:1007500002C0369527950A94E2F721702195292742
:10076000282329272E934F5F5F4F4330510561F7B0
:100770000895682F892F91111CC06530D8F4E8EED8
:10078000F3E040E050E0219130E0062E02C03695C3
:1007900027950A94E2F721703327042E01C0220F17
:1007A0000A94EAF7822B4F5F5F4F4330510559F7A8
:1007B000089580E008959091CC0521E030E0F901A2
:1007C00001C0EE0F8A95EAF7D90102C0AA0FBB1F3C
:1007D0006A95E2F7EA2B01C0220F4A95EAF7892FC2
:1007E0008E23E81303C0892F822B84CF2095822F7C
:1007F0008923FBCF8091960390919503981301C0B4
:1008000008958F5F8770FACF90911705809589239F
:1008100080931705282F2770211110C0891771F0B8
:100820009091CE0592FF0AC08695869586956FDFDA
:100830001092170510921905109218050895982F17
:1008400090958091140589238093140508958091D3
:100850001305811531F01092130510921B051092AB
:100860001A050895803E9105D9F1C8F481339105A8
:1008700009F482C048F48932910509F472C08A32C1
:10088000910509F480C0089589339105E9F0823813
:100890009105D1F08533910509F45EC00895843E39
:1008A0009105D9F148F4823E910539F1833E9105D5
:1008B00049F181EE90E00895863E9105C9F1873EA9
:1008C000910509F43EC008952091CD0523702111B2
:1008D00064C02091CE0523FF14C089E290E0089502
:1008E0002091CD0520FD45C03091CE0530FF09C0D7
:1008F00024FD24C083EE90E008952091CD0522FDD3
:10090000F7CF08952091CD0522FD44C03091CE054A
:1009100030FD43C024FFF5CF11C02091CE0521FF4B
:10092000F0CF8091CD0584FD09C087EE90E0089559
:100930002091CD0523FFE5CF24FFF7CF80E090E0A5
:1009400008952091CD0523FD2BC03091CE0531FFB8
:10095000E1CF84EE90E008952091CD0525FFD1CF21
:10096000BCCF2091CD0525FD1EC02091CE0523FFD3
:10097000C8CF89E390E008952091CD0526FFC1CF2F
:100980008AE290E008952091CD0526FFBACF81E359
:1009900090E0089582EE90E0089580EE90E0089552
:1009A00086EE90E0089585E390E008959091CD055E
:1009B00092FF10C041E0282F2471243009F040E05C
:1009C00031E0282F2871283009F030E0431711F06A
:1009D0002CE0822793FF10C041E0282F247124319E
:1009E00009F040E031E0282F2871283109F030E08B
:1009F000431711F02CE082273091CE0530FF10C054
:100A000051E0282F2171213009F050E041E0282FDA
:100A10002871283009F040E0541711F029E08227AE
:100A200031FF10C041E0282F2171213109F040E051
:100A300031E0282F2871283109F030E0431711F0F8
:100A400029E0822794FD877E08951F93CF93DF933B
:100A500009DFEC01811522E5920708F052C08115EB
:100A600040E5940708F0CDC0803E910520F58D3C0F
:100A7000910508F0A1C0883A910570F4853A910576
:100A800008F097C081309105B9F10497813A91053A
:100A900098F1C0E0D0E030C0885A91094B97C8F770
:100AA000C85AD0E0CC0FDD1FC25CDE4F0990D88160
:100AB000C02DD46421C0811550E49507B0F4C11550
:100AC00080E2D80708F0B3C0C83ED105A8F0CE0137
:100AD0009A9581159F41E8F68D2F68DF182FCE017A
:100AE0009927C0DEEC01D12B07C09927BBDECC27AC
:100AF000DF70C82BD92BD06ACE01DF91CF911F9127
:100B00000895803842E59407C8F5803652E5950788
:100B100008F05BC0C03482E5D807D0F4C03292E55B
:100B2000D90708F04BC08C2F8695869520E2829FCE
:100B3000C0011124C37021E030E0A90102C0440FBC
:100B4000551FCA95E2F7EA01C82BD92BDD68D4CF2F
:100B50008C2F86958695877050E2859FC001112461
:100B6000C37021E030E0A90102C0440F551FCA95AF
:100B7000E2F7EA01C82BD92BDC68BECF803C52E5F6
:100B8000950758F48F71C03AD245A0F590E0982FA0
:100B90008827EC01C46FD06AAFCF805C9245809704
:100BA00008F077CFDC2FCC27CC27DF71C06FD06A5D
:100BB000A3CFA497D064A0CFD0659ECFCF71D0E053
:100BC000DC2FCC27C16FD06A97CF8695869587702A
:100BD00020E2829FC0011124C37021E030E0A9010E
:100BE00002C0440F551FCA95E2F7EA01C82BD92B62
:100BF000DA6882CFDBDEC82FD0E0DC2FCC27D062D2
:100C00007BCF8F71D3DE93E0CC0FDD1F9A95E1F798
:100C1000CC27DF70282F30E084FF05C050E1859F8E
:100C2000900111243327C22BD32BD06965CF8D2F90
:100C30008F71BCDE182FCE01992714DEEC01D12B69
:100C4000DECF80E0089581152CE7920741F42091D2
:100C5000820330918303232B11F480E090E0089508
:100C6000EDE8F4E080E090E063EE74E246E055E207
:100C700028E735E277836683518740873387228769
:100C800097878687019670968830910599F7089521
:100C900010925D0510925C05ECE1F5E08581811113
:100CA00002C014821682379685E0E435F807B1F762
:100CB0000895AC0130915F0560915E05232F6213AA
:100CC00001C00895822F90E0FC01EE0FFF1FEC5A47
:100CD000FA4F0190F081E02DE417F50791F467E0F9
:100CE000649FF001659FF00D1124E45EFA4F41E02E
:100CF00044832313E6CF01968370992780935F0581
:100D000008950196282F2370DACFFC018481862371
:100D100081110AC082818115B9F06823908593FF03
:100D200005C081E061110FC080E00895282F229551
:100D30002F708F70282B962F92959F706F70962B27
:100D400081E02913F1CF089581E00895282F35EB34
:100D50002303C001112497FF04C080589109892FF3
:100D6000089580589F4FFBCF8091ED0380FD14C004
:100D700081FD14C082FD16C08091EC03811581F0C5
:100D80008E3180F420E5829FC00111246EE170E075
:100D90000E94C731862F089584E1089588E208955E
:100DA00088E0089580E508958091ED0380FD17C0E7
:100DB00081FD17C082FD19C08091EB03811599F068
:100DC000883298F428E0829FC001112468E270E024
:100DD0000E94C7316115710551F0862F089562E0B8
:100DE000FCCF64E0FACF61E0F8CF68E0F6CF81E0B5
:100DF0000895FA01309709F009950895E0918B0361
:100E0000F0918C03309739F00190F081E02D30970C
:100E100011F00995089580E00895DC01E0918B03BD
:100E2000F0918C03309759F086819781892B39F0A6
:100E300082E08C930680F781E02DCD01099508951D
:100E4000A3E0B0E0E6E2F7E00C948C319C018091E5
:100E5000DC019091DD0182179307B1F03093DD0141
:100E60002093DC01E0918B03F0918C03309761F0CB
:100E70000084F185E02D309739F083E089833B834E
:100E80002A83CE01019609952396E2E00C94A831BD
:100E9000A3E0B0E0EEE4F7E00C948C319C0180918B
:100EA000DA019091DB0182179307B1F03093DB01F7
:100EB0002093DA01E0918B03F0918C03309761F07D
:100EC0000084F185E02D309739F084E089833B83FD
:100ED0002A83CE01019609952396E2E00C94A8316D
:100EE0009C01FC0132968FEF90E04191461751F042
:100EF0008F3F19F4411101C0892F9F5F9630A9F7E8
:100F00008F3F09F40895280F311D87FD3A95F901A7
:100F100062830895E8EBF1E09191891302C0DF014B
:100F20001E9291E0EE3BF907B9F70895DC01FB0151
:100F300011969C9111978181981322C012968C91E1
:100F40001297811519F0928189131AC013968C910A
:100F50001397811519F09381891312C015968C91FE
:100F60001597811519F0958189130AC014969C91E3
:100F7000911521F081E02481291303C080E001C094
:100F800081E0817008958091010108952FB7F89450
:100F90006091D6017091D7018091D8019091D901CB
:100FA0002FBF0895CF92DF92EF92FF92CF93DF93FE
:100FB000D82FC92FC0908704D0908804E09089046E
:100FC000F0908A04E3DF6C197D098E099F09643F64
:100FD00071408105910510F1D9DF6B017C0182E33D
:100FE00090E0A0E0B0E0C0925202D0925302E092B2
:100FF0005402F092550280934E0290934F02A093B8
:101000005002B0935102D0938504C0938604DF91BF
:10101000CF91FF90EF90DF90CF90089584EF91E013
:10102000A0E0B0E0E0CF87E797E7909301088093D6
:10103000000888E19AE00FB6F894A89580936000C4
:101040000FBE90936000FFCF0895FC019B0180913B
:10105000CC019091CD018617970740F0672B29F4BA
:101060008091E8008E778093E800C90140E0009706
:1010700041F4411106C08091E80082FF2FC080E05A
:101080000895209184032115A9F12530A9F120911B
:10109000E80023FD2DC02091E80022FDECCF209137
:1010A000E80020FFE4CF3091F3002091F200009798
:1010B00019F02830310558F041E02830310509F0A9
:1010C00040E02091E8002E772093E800D0CF4191B6
:1010D0004093F10001972F5F3F4FE9CF8091840348
:1010E000811541F0853041F08091E80083FFC3CF46
:1010F00081E0089582E0089583E008958091C6011B
:1011000087FF13C08091E80082FF06C08091E8004D
:101110008B778093E8000895809184038111F2CF4A
:101120000895809184038115D9F38091E80080FFB0
:10113000F8CF8091E8008E77ECCF2091E4003091D9
:10114000E50095E6A9012091EC00822F817020FF37
:1011500006C08091E80080FF06C080E008952091DD
:10116000E80022FD1AC080918403811589F0853042
:1011700089F08091EB0085FD0FC02091E400309153
:10118000E50042175307F9F29A95E1F684E00895D5
:1011900082E0089583E0089581E00895E8EDF0E0AD
:1011A00080818E7F80831092E2001092DA0010928C
:1011B000E100A0EEB0E08C9181608C9380818F770C
:1011C000808319BCA7EDB0E08C918E7F8C938081D9
:1011D0008F7E80831092C5010895E0918B03F0917A
:1011E0008C03309739F00284F385E02D309711F0AD
:1011F00060E209950895982F9093E900891771F09E
:101200007091EC002091ED005091F00021FD09C09B
:101210009F5F973089F78093E9000895762F242FF8
:1012200050E03091EB003E7F3093EB003091ED00C9
:101230003D7F3093ED003091EB0031603093EB0057
:101240007093EC002093ED005093F0002091EE009D
:1012500027FDDECF0895A0E0B0E0E1E3F9E00C94D3
:101260008631C8EDD0E088818F7E8883E7EDF0E09D
:1012700080818160808384E082BF81E08093C501AA
:1012800088818E7F888302EE10E0F8011082109230
:10129000DA0081EEC82ED12CF601108288818F777A
:1012A000888388818068888388818F7D888319BC42
:1012B000109284031092C40110924B021092C30149
:1012C00090EEE92EF12CF70180818B7F808388815D
:1012D0008160888342E060E080E08DDFF6018081FC
:1012E0008E7F8083F8018081816080838081886027
:1012F0008083F70180818E7F8083888180618883ED
:10130000CDB7DEB7E8E00C94A231E091960390915E
:10131000950329E0E91302C080E00895AE2FB0E004
:101320002E9FF0011124E956FC4F3181361306C07F
:101330003081381303C03581341304C0FD01319668
:10134000E770E8CF81E0089581E08093CF05409178
:10135000CF055091D0056091D1057091D2058FE0F5
:1013600090E00E94473240E050E0BA0183E190E013
:101370000C9447320F931F93CF93DF938B01EA01B5
:1013800090918403943051F58093E9008FEF909110
:10139000E80095FD06C09AE69A95F1F700C08A9597
:1013A000B1F78091E80085FF19C0C7DE811111C037
:1013B0008091E80085FD06C08091E8008E778093DB
:1013C000E800F3CFF80181918F018093F10021971C
:1013D00079F78091E8008E778093E800DF91CF91D4
:1013E0001F910F910895792F603229F440E250E067
:1013F000682F82E0BFCF0895CF93DF93D82FC92FF6
:1014000048E050E0682F792F81E0B4DF88E0ED2FCD
:10141000FC2FAEECB1E001900D928A95E1F7DF91DF
:10142000CF910895BC0146E050E084E0A3CFBC0119
:1014300043E050E084E09ECF9091CE0592FB2227BE
:1014400020F9281771F080FB92F99093CE056091F6
:10145000CD057091CE0584E090E00E944F3282E08D
:10146000D3C908951F93CF93DF93962F122F632F25
:101470008430B0F4911114C0453090F4C42FD0E002
:10148000CC0FDD1F9AE0899FC00DD11D1124CE0124
:1014900089960E943532612FCE018A960E9435329C
:1014A000DF91CF911F910895CF9363E472E084EFB1
:1014B00093E03CDDC82F811519F084EF93E0ADDC9B
:1014C0009091F50386E0E4EFF3E0DF01282F1D9211
:1014D0002A95E9F79093F503A3E4B2E001900D9209
:1014E0008A95E1F781E0911101C080E08C2BCF91CA
:1014F0000895A4E2B0E0EFE7FAE00C948031409167
:10150000F4035091F5036091F6037091F703809115
:10151000F8039091F9039CD42093F4033093F503DE
:101520004093F6035093F7036093F8037093F90325
:1015300086E0E4EFF3E0DE01179601900D928A95C4
:10154000E1F71091F70311951A8786E0FE013796AF
:10155000DE011D9601900D928A95E1F726E0FE01CD
:101560003D96CE010196DC0101900D922A95E1F79E
:1015700026E0FC01A4EFB3E001900D922A95E1F77B
:1015800026E0E4EFF3E0DE01179601900D922A9534
:10159000E1F726E0FE013796DE01539601900D92A9
:1015A0002A95E1F726E0FE017396DC0101900D9289
:1015B0002A95E1F726E0FC01A4EFB3E001900D923B
:1015C0002A95E1F726E0E4EFF3E0DE015F96019073
:1015D0000D922A95E1F76091F6032091FA03D82E37
:1015E000E92EF090F8030091F903211509F46DC07C
:1015F000062E000C770B880B990B0E94023320E01B
:1016000030E040E05EE30E948E3320913E02309154
:101610003F0240914002509141020E946B323B01D7
:101620004C01612F110F770B880B990B0E9402332D
:1016300020E030E040E05EE30E948E3320913A02E9
:1016400030913B0240913C0250913D020E946B322E
:101650005B01C82E192FB301C4010E94CF32062F9F
:10166000B5018C2D912F0E94CF32F62E602F002EC7
:10167000000C770B880B990B0E9402339B01AC0185
:10168000B301C4010E946A3260933E0270933F022C
:1016900080934002909341026F2D0F2C000C770B2A
:1016A000880B990B0E9402339B01AC01B5018C2D74
:1016B000912F0E946A3260933A0270933B028093AA
:1016C0003C0290933D0210E060E069A31AA3FBA2E4
:1016D0000CA386E0FE017F96DE01179601900D9225
:1016E0008A95E1F786E0FE013796AD2DBE2D01907B
:1016F0000D928A95E1F786E0ED2DFE2DDE015996DB
:1017000001900D928A95E1F786E0FE017996DE015F
:10171000179601900D928A95E1F786E0FE013796C3
:10172000A4EFB3E001900D928A95E1F786E0EEEE2A
:10173000F3E0DE01179601900D928A95E1F7809112
:10174000F5039885892B8093F503AEDE811102C0E5
:101750008091420210924202A496EEE00C949C31D9
:101760000F931F93CF93DF93843008F561111FC04F
:101770004530E8F4C42FD0E0CC0FDD1F2AE0829F73
:10178000C00DD11D1124CE0189960E941432082F5C
:1017900010E0102F0027CE018A960E941432980183
:1017A000282BC901DF91CF911F910F91089580E0FF
:1017B00090E0F8CF462F2091870330918803232BA8
:1017C00089F4703F39F4603F69F48091850390910A
:1017D00086030895711106C0653020F4843010F43A
:1017E00060E0BECF80E090E00895A0E0B0E0EBEFD5
:1017F000FBE00C9487317C010091CC058091CB05F6
:10180000082BC3E0D0E010E0C8010C2E02C0959573
:1018100087950A94E2F780FD09C02197A8F7D12C9B
:101820008D2DCDB7DEB7E7E00C94A331DC2EB701E8
:101830008C2FC0DF0AD9019781F3F2CF0F931F934A
:10184000CF93FC0187819085009789F48581008181
:101850001181811581F0611571F0C801C6DFC82FB3
:10186000682FC8010E949503B8018C2FA3DFCF9188
:101870001F910F910895C8010E94B903C82FF4CF9A
:10188000CF93DF93D82FC92FB0DF6D2F7C2F92DF3E
:10189000DCD8DF91CF910895FC0184818115A9F0F6
:1018A00087819085009799F0D0D8282F92959F70C6
:1018B0009630B9F080F4925F9F70923030F4203F00
:1018C000D1F058F481E0283E58F080E008958081FE
:1018D0009181D6DFEACF9A5FEFCF81E0243FA9F76D
:1018E000089591E0813F09F090E081E0283E08F002
:1018F00080E0892B089581E00895382F292FCB01AE
:10190000A32FB22F8F3A22E09207A105B10520F450
:101910008F5A9E4F0C94143280E0089585E290E037
:101920000E941432823D89F486E290E00E941432D3
:10193000893759F487E290E00E94143291E08734AD
:1019400009F090E0892F8170089580E0FCCFAAE033
:10195000B0E0EDEAFCE00C948631C0908203D090B8
:10196000830381E090E0909383038093820310E0EF
:1019700082E0E82E83E0F82E00E021E030E0111153
:1019800004C0F701859195919C01402F60E0812F63
:1019900069DD0F5F82E0E80EF11C053071F71F5F13
:1019A000143031F71A8219821C821B821E821D821A
:1019B00018861F8288EC90E09A87898701E610E0FC
:1019C000FE0131967F014AE050E0B801C7010E9454
:1019D0005332065F1F4F013B1105A9F78AE0F7015B
:1019E00011928A95E9F74AE050E0B801C7010E94D8
:1019F0005332065F1F4F01301007A9F789E0F70146
:101A000011928A95E9F78FEF9FEF9E838D8387E090
:101A10008A874AE050E0B801C7010E945332065F4E
:101A20001F4F0135F1E01F07A1F7D0928303C09249
:101A300082032A96E8E00C94A231AAE0B0E0E3E247
:101A4000FDE00C948631E0EEF1E080E5DF011D92CF
:101A50008A95E9F7ECE1F5E088E3DF011D928A95CC
:101A6000E9F780EEC82E81E0D82E7F0101EB10E06F
:101A7000F701D182C0824AE050E0B801CE01019660
:101A80000E94043288E0FE013196D60101900D9249
:101A90008A95E1F789859A85D70113969C938E9351
:101AA0001297BAE0CB0ED11CE7E0EE0EF11C065FF8
:101AB0001F4F01301007E1F62A96E8E00C94A2319E
:101AC000AAE0B0E0E6E6FDE00C9484310AE014E020
:101AD000EE24E394FE2C97E0B92E2FEDC22E21E0E8
:101AE000D22EAA24A3944AE050E0B701CE01019679
:101AF0000E940432F8013896DF018B2D1D928A95E1
:101B0000E9F789819A81D80111969C938E938F81F0
:101B100012968C9312978D8113968C9313978885C8
:101B200014968C931497898515968C9315978B81B1
:101B30009C8117969C938E9316978A8587FD04C087
:101B40001E96DC92CE921D9780FF02C0F801A086FF
:101B500081FF07C0D80118969C911897926018963B
:101B60009C9382FF04C0F80190859460908783FF66
:101B700007C0D80118969C911897986018969C9366
:101B800084FF04C0F80190859061908785FF07C0AD
:101B9000D80118968C911897806218968C93BAE0A9
:101BA000EB0EF11C015F1F4FE1E5EE16E1E0FE06D2
:101BB00009F099CF2A96EAE00C94A031282FCB01A6
:101BC000283070F44AE0249F90011124B9016F5924
:101BD0007F4F4AE050E00E94043280E090E0089598
:101BE0008FEF9FEF0895AAE0B0E0E9EFFDE00C94DD
:101BF0008C319C0197558115914068F4BE016F5F4F
:101C00007F4F822FDBDF892B31F489859A852A96D5
:101C1000E2E00C94A83188EC90E0F9CFA0E1B0E0CC
:101C2000E4E1FEE00C947E31FE01319680E1DF01BB
:101C30001D928A95E9F70BE210E091E5A92EBB24ED
:101C4000B3942FEA422E22E0522E612C712C4F01C8
:101C500073016201B1E14B165104610471041CF07F
:101C600080E1C82ED12CA601B501C4010E94263204
:101C7000AC0CBD1C0D2C000CEE08FF084C185D08C8
:101C80006E087F080150104019F76096E0E10C944F
:101C90009A316FEF85E290E00E9435326FEF86E275
:101CA00090E00E9435326FEF87E290E00E9435327B
:101CB00060E088E290E00E94353249DEAFDF62EDFD
:101CC00085E290E00E94353269E786E290E00E946A
:101CD000353267E487E290E00C943532CF9324E00C
:101CE00030E043E060E080E30E94D530C82F8111EE
:101CF00005C00E944A318C2FCF91089582E08A95C9
:101D0000F1F700C0F8CFCF93C82FE8DF8115C9F0F5
:101D10008C2F0E94E7308FE391E00197F1F700C02C
:101D200000000E94FF30C82F92E09A95F1F700C0A2
:101D30000E944A3182E38A95F1F700C08C2FCF913F
:101D40000895C0E0FBCFA2E0B0E0E9EAFEE00C9429
:101D50008931182FF62EC2DF082F811106C000E04E
:101D6000802F2296E5E00C94A531103511F01092E9
:101D7000380210681983FA8262E070E0CE010196A1
:101D80000E941731892B59F78DE58A95F1F70000EC
:101D90000E944A3181E291E00197F1F700C0000012
:101DA000DFCF60E08436910550F067E784342FE29E
:101DB000920728F464E670E00E94B33161508FE02E
:101DC000C2CF0E9440308ADF811509F440C02AE664
:101DD0002A95F1F700C00E944A318AE68A95F1F708
:101DE00000C06AE58AE3AFDF811589F19FE728E348
:101DF00081E0915020408040E1F700C0000082E087
:101E000082DF83E080DF84E07EDF85E07CDF86E0C8
:101E10007ADF0E944A318FE19EE40197F1F700C01A
:101E200000006FE08FE08FDF8FEC97E00197F1F714
:101E300000C0000060E080E186DF64E181E183DFD3
:101E400062E083E680DF80E05EDF8FE35CCF0895B1
:101E5000A8E1B0E0EEE2FFE00C948A314B8B5C8BA2
:101E60006D8B7E8B8F8B988FFE01379686E0DF011E
:101E70001D928A95E9F7809138028F01811108C07F
:101E800060E080E560DF811539F181E08093380200
:101E900025DF811509F180E50E94E730BDE5BA959F
:101EA000F1F7000066E070E0C8010E9430318F81D8
:101EB00087708111109238020E944A3189859A8573
:101EC0009195819591099A8789878B859C859195B4
:101ED000819591099C878B8786E0FE013796DE010C
:101EE000119601900D928A95E1F786E0FE013196F8
:101EF000DE011D9601900D928A95E1F78D8583FD97
:101F000005C0898187FD17C01092390286E0FE0165
:101F10007396DE01179601900D928A95E1F72F8155
:101F2000388549855A856B857C8580E090E0689688
:101F3000E4E00C94A6314B815C812D813E8180913F
:101F40003902811103C081E080933902842F403827
:101F500051054CF08FE78D8B822F2038310544F0EE
:101F60008FE78E8BD3CF40385F4FACF780E8F3CF4D
:101F700020383F4FB4F780E8F4CF1F921FB61F926E
:101F800011248F939F93AF93BF9380914A02811145
:101F900013C08091D6019091D701A091D801B09142
:101FA000D9014196A11DB11D8093D6019093D7010F
:101FB000A093D801B093D901BF91AF919F918F9118
:101FC0001F901FBE1F9018952FB7F8948091D601CF
:101FD0009091D701A091D801B091D9012FBF089558
:101FE000CF93DF93C091140580911605C82B809183
:101FF00013058115F1F0E8DF20911A0530911B05DA
:10200000821B930B8838934110F00E942704D091D3
:10201000130520E088EB91E0FC013081019631113D
:102020002F5F31E08E3B9307B9F721110E942704FF
:10203000CD2B8091090480958C2390910804892BE5
:102040008093B60148E050E06DE873E086EB91E0E4
:102050000E94F031892BB9F088E0E6EBF1E0ADE8C1
:10206000B3E001900D928A95E1F7E0918B03F09136
:102070008C03309741F00280F381E02D309719F006
:1020800086EB91E00995DF91CF910895811531F0AC
:1020900090911405892B80931405A2CF0895811582
:1020A00019F00E941F049CCF0895811531F0909182
:1020B0001605892B8093160593CF0895811539F065
:1020C00080959091160589238093160589CF0895F0
:1020D000CF93DF93EC014A855B856E857F850E94F7
:1020E000F9069B81909580911605892380931605AA
:1020F0008C810E941F0474DF86E0FE0111928A9594
:10210000E9F7DF91CF910895CF93DF93EC018D81B3
:1021100081FD16C082608D83809116059B81892B7D
:1021200080931605809114059C81892B809314055A
:1021300057DF488559856E857F85CE010E94F90657
:1021400010920E0510920D058D8180FD02C0CE010A
:10215000BFDFDF91CF910895962F2091CE0522FF0A
:102160000FC0682F660F660F660F692B6093170507
:102170000E947D0329DF9093190580931805089527
:102180000C947D0390911305292F2823211559F0D4
:102190008095892380931305811531F015DF809395
:1021A0001A0590931B05089580E090E0F8CF0CDFAE
:1021B0002091F0033091F103232B211521F080931E
:1021C0007A0390937B032091F2033091F303232B46
:1021D000211521F080937803909379038EEE93E09C
:1021E0000C940D07611509F45DC0E3E3E80FE331DA
:1021F00050F4F0E0ED50FC4C0C94DA310E94B4063F
:1022000081958093F103D3CF0E94B406FACF0E9448
:10221000B40681958093F003F6CF0E94B406FACFFE
:102220000E94D4068093F203EECF0E94D4068195DB
:10223000F9CF0E94D40681958093F303E4CF0E94E6
:10224000D406FACF282F215D330BA90121E030E01D
:1022500001C0220F4A95EAF79091EF03922B9093D9
:10226000EF034091F503815D21E030E0F90102C008
:10227000EE0FFF1F8A95E2F7CF01611509F48CC0BC
:10228000842B8093F50310C98091ED0381608093C6
:10229000ED03B9CF8091ED038260F9CF8091ED031A
:1022A0008460F5CF9091F003482F50E08D3C59F4B5
:1022B0002091F10327FF0DC01092F10391110BC083
:1022C0001092EC0308C08E3CB1F42091F103121679
:1022D0009CF39115B1F09091F2032091F303922BAE
:1022E000911102C01092EB03415D51094830510534
:1022F00008F4B7CF88CF8F3C39F497FFEACF10921C
:10230000F0039091F103DACF803D19F41916BCF374
:10231000E0CF2091F203893D29F41216D4F61092F1
:10232000F203D7CF8A3D19F427FFD3CFF8CF2091FE
:10233000F3038B3D29F427FFCCCF1092F303C9CFD1
:102340008C3D19F41216CCF3C4CF2FE2280F28309D
:1023500080F4FA01E15DF10921E030E001C0220FD3
:10236000EA95EAF720953091EF0323232093EF03BA
:10237000B0CF2091ED032E7F8D3D59F02091ED03DC
:102380002D7F8E3D31F08F3D09F0A3CF2091ED03DD
:102390002B7F2093ED039DCF8095842372CFCF9325
:1023A000C82F8115A9F08CEF8C0F813A98F4E8EBD7
:1023B000F1E08EEB91E02191C21709F43DC08E1738
:1023C0009F07C9F76C2F86EB91E00E94700708DE2B
:1023D000CF91089580E28C0F883068F4C77021E0B7
:1023E00030E001C0220FCA95EAF780911405822BD4
:1023F00080931405ECCF8BE58C0F833038F42C2FB1
:102400002452330BC9010E942007E2CFE8E5EC0F0C
:10241000EB3150F4F0E0EE0FFF1FEC58FE4F8081DF
:1024200091810E944807D4CF83E38C0F833180F6DB
:1024300061E08C2FD7DECCCF8C2F0E948A07D0DDB5
:10244000C1CFCF93DF93EC01805E9109089720F014
:1024500065E570E1209711F466E470E1CE010E9419
:102460006E038C2F9CDFDF91CF910895811559F178
:102470009CEF980F913A18F40E948A07B1CD90E230
:10248000980F983050F4877091E001C0990F8A95A9
:10249000EAF7892F0E941F04F1CF9BE5980F933034
:1024A00020F480E090E00C94200798E5980F9B3191
:1024B00020F480E090E00C94480793E3980F933168
:1024C00010F460E08FCE08951F93CF93DF93182F01
:1024D000EB0165DF209731F4812FC8DFDF91CF91C9
:1024E0001F9108958FEC97E00197F1F700C000006D
:1024F0002197F0CF60E570E0893311F060E070E083
:10250000E3CFA0E0B0E0E7E8F2E10C948531EC0124
:1025100088818115D9F0813009F03FC089818130EF
:1025200021F48A812396E6DFF3CF823021F48A8179
:10253000239635DFEDCF833021F48A81239696DF11
:10254000E7CF843041F022968111E2CFCDB7DEB7DC
:10255000E9E00C94A1318A81239620E030E09AE0F2
:10256000682F6053770BAB016A30710560F021155D
:10257000310551F3EFECF7E03197F1F700C00000BF
:1025800021503109F4CF929FB001939F700D112417
:102590009A01260F371F8991E3CFE82FF0E0E3542B
:1025A000FE4FB490282F26952695269530E0F90108
:1025B000E355FE4FE4908770F12C082E02C0F5948D
:1025C000E7940A94E2F7E0FAEE24FF24E0F8F90138
:1025D000E356FE4FC490D12C082E02C0D594C79468
:1025E0000A94E2F7C0FACC24DD24C0F8F901E357DD
:1025F000FE4F049110E002C0159507958A95E2F709
:1026000001701127E114F10411F081EEC8DEC1144C
:10261000D10411F086EEC3DE60E070E08B2D54DF54
:10262000C114D10411F086EE21DFE114F10411F0A0
:1026300081EE1CDF0115110511F08CE25BDF2196A4
:1026400067CF1F93CF93DF93182FA0918304B0918E
:102650008404109709F449C01092860410928504EE
:1026600010920904109208041696CD91DC911797E8
:10267000CE019A9581159F4108F4D07ED1E0C11119
:1026800001C0D0E01996ED91FC911A97309731F086
:102690001B966D917C9180E00995D823D11539F076
:1026A0008CEF8C0F813A28F58C2F0E948A07111528
:1026B000A9F0E0918304F0918404808584FD0EC02C
:1026C00080918204811551F0808191819C0121507B
:1026D00031092F333E4710F40E94D20781DC10925B
:1026E00084041092830410928204DF91CF911F9191
:1026F000089576DC8C2FBADEDACFCF9310921405D2
:10270000C6E0E8EBF1E0DF018C2F1D928A95E9F736
:1027100080E090E00E94200780E090E00E9448075F
:10272000109216055DDCEEEEF3E0DF011D92CA9516
:10273000E9F71092EC031092EB031092ED0337DDF2
:10274000CF910895DADF2FE78AE196E021508040AB
:102750009040E1F700C0000088E19AE00FB6F894DD
:10276000A895809360000FBE90936000FFCFAAE20F
:10277000B0E0EDEBF3E10C948B3186EC91E0FC01E1
:1027800001962091F100208321E08E3C9207B9F759
:102790008091C701893009F459C0C8F4823009F426
:1027A000B6C0833009F485C0813089F18091E8009A
:1027B00083FFEAC08091C6019091C7019A3008F06A
:1027C000E3C0E92FF0E0EA5FFB4C0C94DA318A3089
:1027D00009F48CC08B3051F78091C601813231F7FA
:1027E0008091CA019091CB01892B01F78091E8007B
:1027F000877F8093E8000E947E0881E09091C80165
:10280000911101C080E08093020177DFCFCF8091EA
:10281000C601813A59F68091E800877F8093E800ED
:102820008091CA019091CB01892B61F060E080E03A
:1028300090E070E00E9425088091E8008B778093FB
:10284000E800B4CF68E08EEC91E0F3CF8091C60150
:10285000813209F0ABCF8091CA019091CB018D7F7D
:10286000892B09F0A3CF8091E800877F8093E8004F
:102870008091E80082FF18C09091F3008091F200EF
:10288000029731F48091F100813011F0863021F40B
:102890008091F100809301018091E8008B77809313
:1028A000E8000E947E0882CF809184038111E0CFEE
:1028B0007DCF8091C601813A09F078CF8091CA011D
:1028C0009091CB01892B09F071CF8091E800877F2F
:1028D0008093E8008091E80080FFFCCF80910201A6
:1028E0008093F1008091E8008E77D9CF8091C60166
:1028F000813209F05BCF8091E800877F8093E80008
:102900000E947E088091C901809300014FCF809181
:10291000C601813A09F04ACF8091E800877F809311
:10292000E8008091E80080FFFCCF80910001D8CFC3
:10293000803889F0823841F58091CA018F708730E4
:1029400018F58093E9008091EB0085FB882780F9DA
:102950001092E90006C080914B02880F9091C3014C
:10296000892B9091E800977F9093E8008093F10085
:102970001092F1008091E8008E7723C0811116C07B
:102980008091C801813011F18091E80083FF0AC075
:102990008091E800877F8093E8008091EB0080625F
:1029A0008093EB00AA96E3E00C94A731823061F7A4
:1029B0008091C801811589F01092E9008091E800AA
:1029C000877F8093E8000E947E08DECF81E093300D
:1029D00009F080E080934B02EFCF8091CA018F70A5
:1029E0002FEF280F263080F68093E9002091EB002E
:1029F00020FFE2CF933031F48091EB00806280932E
:102A0000EB00DACF9091EB0090619093EB0021E026
:102A100030E0A90102C0440F551F8A95E2F74093A8
:102A2000EA001092EA008091EB008860E8CF811103
:102A3000ABCF1091C8011F778091E3008078812B84
:102A40008093E3008091E800877F8093E8000E94F4
:102A50007E088091E80080FFFCCF8091E3008068D1
:102A60008093E30083E0111101C082E0809384032E
:102A70008BCF8058823008F087CF8091C801909129
:102A8000C9018C3D53E0950799F583E08A838AE27A
:102A900089834FB7F894DE01139620E03EE051E2BF
:102AA000E32FF0E050935700849120FF03C08295FC
:102AB0008F703F5F8F708A30C8F0895C90E08D9393
:102AC0009D932F5F243161F74FBF8091E800877F8E
:102AD0008093E8006AE270E0CE0101960E9425082A
:102AE0008091E8008B778093E8004ECF805DE6CF41
:102AF000292F33272330310509F44EC078F52130D2
:102B0000310509F488C08BE590E0EDE3F2E0223076
:102B1000310509F039CF2091E800277F2093E800A4
:102B20002091CC013091CD018217930708F49C01CC
:102B300040E02115310509F073C0411171C0809149
:102B4000E80082FDCDCF80918403811549F2853064
:102B500039F28091E80083FFF2CFC2CF8091CA01A1
:102B60009091CB012132310509F446C02232310562
:102B700009F00ACF8330910508F006CFFC01EE0F73
:102B8000FF1FE35DFE4F0190F081E02D865D9E4FBB
:102B9000DC018C9190E010C09C013327823021F140
:102BA0002330310568F4232BB9F4EEEFF2E0E49121
:102BB0008E2F90E0EEEFF2E0009709F4E5CEABCF78
:102BC0002330310509F0E0CEEAEAF2E0E4918E2FFD
:102BD00090E0EAEAF2E0F0CFEEEEF2E0E4918E2F40
:102BE00090E0EEEEF2E0E8CFE8ECF2E0E4918E2F38
:102BF00090E0E8ECF2E0E0CF8330910508F0C4CE3D
:102C0000FC01EE0FFF1FED5CFE4F0190F081E02D07
:102C100089E090E080CF82E190E0E8E9F2E07BCFCC
:102C200080918403811509F45BCF853009F458CF76
:102C30008091E80083FD54CF8091E80082FD7FCF32
:102C40008091E80080FF75CF9091F3008091F200B1
:102C50002115310519F08830910550F041E00897B1
:102C600009F040E08091E8008E778093E80061CF22
:102C700044914093F1003196215031090196E8CFFB
:102C8000803809F081CE8091E800877F8093E8004A
:102C90008091C4018093F1006DCE811175CE1091A9
:102CA000C801123008F070CE8091E800877F8093D1
:102CB000E8001093C4010E947E081115F9F084E029
:102CC0008093840342E061EC81E00E94FB0842E2D1
:102CD00061EC84E00E94FB0842E261EC82E00E9429
:102CE000FB0842E260EC83E00E94FB0880918403D1
:102CF000843051F482E08093030146CE8091E3005A
:102D000087FDDDCF81E0DCCF81E0F5CFA0E0B0E052
:102D1000ECE8F6E10C948731162FD72FC42FD22E72
:102D2000811599F0409311054FD99093C20180937A
:102D3000C101C77081E001C0880FCA95EAF7A6D922
:102D4000CDB7DEB7E7E00C94A3319091110549139C
:102D500033C0E090C101F090C20136D99C012E1918
:102D60003F097901812F9D2F0E94F30DE816F90686
:102D700018F5D0E2DD0DCD1591F0C77011E0812F6F
:102D800001C0880FCA95EAF78AD9D83040F48D2D52
:102D9000877001C0110F8A95EAF7812F77D9802FAC
:102DA000A9DBD83068F62D2D277081E001C0880F8F
:102DB0002A95EAF774D9C4CFC77081E001C0880FA3
:102DC000CA95EAF7F7CFACE0B0E0E9EEF6E10C9493
:102DD0007D317C01DC0114968C91811509F4E2C1EE
:102DE00061E0C7010E941E0C8C01F70185818115ED
:102DF00029F180910D0590910E050097F9F00817C3
:102E00001907E1F0FC01FF27887F9927892B09F03A
:102E1000A7C0A4E0EE0FFF1FAA95E1F7E357FB4F11
:102E200085818460858311830083CF016DD91092E1
:102E3000160561E0C7010E941E0C8C01D7018C9120
:102E4000813069F411968C91811109C0BDD890939D
:102E5000FD038093FC03F70185818093FB03D70179
:102E600015968C910115BEE71B0709F07CC08115F2
:102E700009F18091CF0590E0019665E070E00E9435
:102E8000B3318093CF054091CF055091D00560912B
:102E9000D1057091D2058FE090E00E944732E09119
:102EA000CF05F0E0EE0FFF1FE655FE4F80819181C8
:102EB0000E94D10ED70115968C91811163C06801D3
:102EC000A7E5DA1AC114B1E0DB0668F56EEF73E02E
:102ED0008C2D0E94DE0D892B31F5C60154E0880F40
:102EE000991F5A95E1F7FC01E357FB4F22812130EE
:102EF00009F02FC12091FE033091FF03232B99F09D
:102F00002091000430910104232B69F020910204E8
:102F1000309103044091040450910504242B352B77
:102F2000232B09F420C1F7013580311409F43EC187
:102F30000E35FCE71F0709F421C10F352CE71207F6
:102F400051F00D353CE7130709F030C180911001B5
:102F5000811509F413C11092100180E072DB11C1D8
:102F6000E0E0F0E05DCF0130EEE71E0709F0A2CF10
:102F7000811509F49FCF8091FA0391E0892780930E
:102F8000FA0398CFC80197578038910560F6003151
:102F900008F0F7C06EEA72E080E090E00E947D0CDD
:102FA0008111EFC0812C912C5401011146C004E025
:102FB0009E012F5F3F4F6901D601E02F1D92EA95D8
:102FC000E9F724013501FFEF4F1A5F0A6F0A7F0A04
:102FD000C501B4010E947D0C8983811509F4D1C01B
:102FE000813009F0B3C0A50194012E5F3F4F4F4FD0
:102FF0005F4F2D833E834F835887C301B2010E94E8
:103000007D0C182F8A83811509F4BBC08FEF810FC7
:10301000833078F56D817E818F8198850E947D0C4B
:103020008B83811511F0C6016CDA2401350133E080
:10303000430E511C611C711C19C0BFEA8B16B2E013
:103040009B06A104B10409F49CC0C501B4010E940F
:103050007D0CEFEF8E1A9E0AAE0ABE0A8111EDCFEB
:103060000150A3CF4D805E806F8078845301420170
:10307000A3CF8BEF810F8330A0F52401350143E00E
:10308000440E511C611C711C6D817E818F8198855D
:103090000E947D0C8B83811549F3C301B2010E940C
:1030A0007D0C8C83811108C02401350154E0450E4C
:1030B000511C611C711CDACF8B819C818130AFEF78
:1030C0009A0710F0982F8827163029F0173031F022
:1030D0000E94D824E9CF0E948524E6CF0E94A6242E
:1030E000E3CF143009F0BECF6D817E818F8198854A
:1030F0000E947D0C182F24013501B4E04B0E511CA9
:10310000611C711CC501B4016D5F7F4F8F4F9F4FD4
:103110000E947D0C1115A9F1811599F18150990B2F
:103120004FEF489F9001499F300D1124E12FE1504E
:10313000FF0B2E0F3F1F2150310908F497CF8FEC62
:1031400097E00197F1F700C00000F5CFC601D9D98B
:103150008DCF223009F0E7CE209102043091030494
:10316000232B09F4E0CEFC01EE56FB4F20812E7F8D
:10317000208383579B4F0E948410D5CE81E080939B
:103180001001809117058770811561F0D7011596A0
:103190008C91811539F08091CE0582FF03C082E0C9
:1031A0000E9404042C96E1E10C9499318091100165
:1031B000811168C0C80197558115914008F0FDC084
:1031C0005801F8EFAF22BB24A114B104D1F6F801E5
:1031D000FF2734E0EE0FFF1F3A95E1F79F012357D9
:1031E0003B4F6901D70115968C91EE56FB4F9081AC
:1031F00080FB90F99083811509F4D8C10E94E40FF7
:103200009093100580930F05F60182818F5F828372
:103210008091160590911405892B83838091130565
:1032200084834681578166857785C6010E94F906A9
:10323000D60115968C9181FF5801B0920E05A0928F
:103240000D05D70115968C91811509F4A7C510922B
:103250001105980130572332310508F088C584E004
:1032600090E00E9421329093CE058093CD05F80125
:10327000E150F047E232F10508F0E0C1E05FFB4CBD
:103280000C94DA31380150EE651A7108509015052A
:1032900080911405582A80911305582A88E06816F1
:1032A000710408F05EC098012770332781E090E038
:1032B00001C0880F2A95EAF7311409F44FC0582A43
:1032C000D7018D919C910E94B90321E030E0F90172
:1032D00002C0EE0FFF1F8A95E2F7FE83ED83209177
:1032E0008304309184043A87298740918B0450915C
:1032F0008C045C874B874AE0C42E44E0D42EA12C7A
:10330000B12C511005C0D60112968C9181111BC0B1
:10331000F601838190E02D813E8182239323892BC6
:1033200091F08085982F9770911101C087E038E067
:103330006316710408F065C0311409F45EC0869507
:103340008170811163C09FEFA91AB90AAFE0CA0E5C
:10335000D11CB8E0AB16B104A1F61CC08095582270
:10336000AFCF311037C080918B0490918C04081737
:10337000190781F410928C0410928B041092870428
:10338000109288041092890410928A041092860484
:10339000109285048091830490918404009709F42D
:1033A00009CFE8E06E16710408F0EBC0652D0E94AD
:1033B0008506811102C081E044D9F7018581F801B9
:1033C000E851FC47E730F10508F03BCFEE5CFB4CE1
:1033D0000C94DA3110938C0400938B040E94C6077E
:1033E00060938704709388048093890490938A047F
:1033F000109286041092850463CF82FB882780F99F
:10340000A0CF311409F49FCF80FF9DCFD6018D90BE
:103410009C900815190519F4311409F494CFE98525
:10342000FA85EC15FD0509F48ECFD6011D96ED91B8
:10343000FC91309721F08081811509F484CF652DAE
:10344000C6010E948506811509F47DCF81E008152B
:10345000190509F080E0482E43208114910441F0C1
:10346000411006C0EB85FC858E169F0609F06BCFD8
:1034700080E0E7D8D0928404C092830481E08093F6
:1034800082048FE08A9DF0018B9DF00D1124E65F90
:10349000FB4F85818093090441100EC08114910473
:1034A00059F0808191819C0124503109213A3105E4
:1034B00008F049C00E948A078FE08A9DF0018B9D29
:1034C000F00D1124E65FFB4FC680D780C6019A95A8
:1034D00081159F4110F420EED22299249394C601C5
:1034E00001978F339E4708F0912C8FE08A9DD00181
:1034F0008B9DB00D1124A65FBB4F1996ED91FC91E9
:103500001A97309731F01B966D917C9181E0099567
:1035100098229114A9F08FE08A9DF0018B9DF00D07
:103520001124E65FFB4F868197810E9444038093BC
:103530000804C60148E06416710440F40E94D207F2
:103540000E94F00F0CC00E943612B6CF0497813A49
:10355000910558F46C2D86EB91E00E9470074114A0
:1035600009F428CE0E94F00F0CCE0E94F00F8FE1DC
:103570009EE40197F1F700C000008C2D0E94CF114E
:10358000EECFDC012D913C910217130739F4311075
:1035900008C01092820480E054D80CCE311409F493
:1035A00009CEFC01808585FD05CEF5CFF901448566
:1035B000558566857785C9010E94F906D60115965D
:1035C0008C9181FF3ECEC6010E94681080910D054E
:1035D00090910E050817190709F033CE10920E05C9
:1035E00010920D052ECE06E221EE41EE6AE17CE757
:1035F0008DDBC7CD07E225EE45EE6BE17CE7F8CF2A
:1036000006E221EE40EE68E17CE7F2CF07E225EE2C
:1036100044EE69E17CE7ECCF06E221EE42EE6CE19C
:103620007CE7E6CF07E225EE46EE6DE17CE7E0CFF2
:1036300008E221E045EE6EE17CE7DACF8091CD052E
:1036400081608093CD056091CD057091CE0584E0B9
:1036500090E00E944F3251D894CD8091CE05886081
:103660008093CE05F0CF8091CD058260EACF809126
:10367000CD058460E6CF8091CD058860E2CF809152
:10368000CE058160EDCF8091CE058260E9CF80913B
:10369000CD058061D6CF8091CD058062D2CF80915B
:1036A000CD058064CECF29D88091CD058068C9CF63
:1036B0008091CD058C60C5CF8091CE058360D0CF41
:1036C0008091CD058E7FBDCF8091CE05877FC8CFFD
:1036D0008091CD058D7FB5CF8091CD058B7FB1CF0A
:1036E0008091CD05877FADCF8091CE058E7FB8CFFD
:1036F0008091CE058D7FB4CF8091CD058F7EA1CFF7
:103700008091CD058F7D9DCF8091CD058F7B99CF09
:103710000E947D138091CD058F7793CF8091CD0549
:10372000837F8FCF8091CE058C7F9ACF8091CD05FE
:10373000992782FF939590FB82F990FB83F981CFC3
:103740008091CE05982F909590FB80F990FB81F9A0
:1037500087CF9091CD05892F8F7B96FF806471CFA5
:103760000E947D139091CD05892F97FB87F9805892
:1037700068CF61E08EE090E00E94353264CF60E077
:10378000F9CF9091CD05892F8F7E94FF806159CF1D
:103790009091CD05892F8E7F90FF816052CF9091BF
:1037A000CE05892F877F93FF88605ACF89E201C3B6
:1037B0000737BCE71B07F9F00837ECE71E0751F1A4
:1037C0009801205E32452032310550F581113FC00D
:1037D0000F7181E090E09C0102C0220F331F0A9517
:1037E000E2F78901622F83E090E00E943532802F5A
:1037F0000E947703C6CC811549F081E00E947D03C9
:1038000043E062E081E00E94DB03BBCC81E00E94E8
:103810008703F6CF811511F082E0F0CF82E0F7CF79
:103820008115A9F00A353CE7130709F476C008F0C2
:103830004EC001305CE7150709F46DC003308CE71A
:10384000180709F462C001151C4709F451C0F701BB
:1038500087819085009709F464C00E9425058C013A
:10386000F701B580A680A2942FE0A22280911705CF
:103870008770811501F1CB2CB114F1F0812F807F7D
:10388000803461F080E2800F8830A8F0812F807E44
:10389000803221F4023078F0A11469F08091CE05D5
:1038A00082FF09C082E00E9404048091170587709E
:1038B000CC24C3948111C12CE12FE295EF70103C10
:1038C00008F0A5C0F0E0E75CFB4C0C94DA310B3556
:1038D000ACE71A0721F18091CE05002482FF039402
:1038E000802D0C351C4709F0B2CF0E941C0AAFCFC7
:1038F0000E947D13EFE7FAE126E0E150F04020401E
:10390000E1F700C000000E9413086FEF7FEF80E036
:1039100090E00E944F320E94A21381E0E6CF80E047
:10392000E4CF8581C080D180811569F0C6010E94F5
:10393000F50B182F682FC6010E949503B601812F41
:103940000E94DA0B8ACFC6010E94B903182FF6CF66
:10395000F12FFF70DF2E103118F0D29490EFD922A2
:10396000B114B9F0D11469F080E2800F883010F002
:10397000011109C0809114058D29809314050E94BE
:10398000F00F802F42C0809116058D298093160577
:10399000F6CF802F0E943612D114C9F180E2800F39
:1039A000883010F0011104C08D2D0E941F0406C044
:1039B000D094809116058D21809316050E94F00FFA
:1039C00026C0212F2F70D22E107F103219F0D294E2
:1039D00080EFD822011549F0013009F484C0B114F8
:1039E00009F490C0A114B1F1CCCF8091CE0582FD35
:1039F0002DC0B11429F1D11439F0809114058D290D
:103A0000809314050E94F00F80E00E94CF11C11432
:103A100009F4D8C08091170580FDD4C0D701159650
:103A20001C928695869586950E947D03C701CBD909
:103A3000809117058695869586950E948703C2C05A
:103A400080E00E943612D11411F3AECFB11469F1A7
:103A5000A11004C08D2D0E944610D9CF31E0A312D1
:103A600010C0109113058D2D8123D81681F20E946C
:103A7000E40F90931B0580931A051D2910931305DD
:103A8000C6CF45E0A412C3CF8D2D0E9446108D2DC8
:103A90000E94C210809115059D2D9823D91609F416
:103AA000B6CF8D2980931505B2CFA11012C08D2DF0
:103AB0000E944F108D2D0E94C210809115059D2DE2
:103AC0009823911509F4A3CFD094D822D09215054C
:103AD0009ECF51E0A5129BCF809114058D218115B9
:103AE00009F495CFE4CFB11429F086E0A81608F0C8
:103AF0008ECFB0CF95E0A91608F089CF8D2D0E940A
:103B00004F1085CFA114D1F3093349F4AFEFB3EFD0
:103B1000E1E0A150B040E040E1F700C00000802F9C
:103B20000E94361274CF812F8695869583708115F9
:103B300061F0813009F06BCFC8019370B11002C001
:103B400080E090E00E94480762CFC8019370B110F6
:103B500002C080E090E00E94200759CF6B2D802F9B
:103B60000E94F21054CF812F8370811138C0B110A0
:103B700027C0402F429546954770440F440F802F31
:103B80008F70042E01C0880F0A94EAF7202F20714D
:103B900004FF07C02FE030E001C0220F4A95EAF78A
:103BA00020951695169513701230A1F0133081F000
:103BB0003091CB05113059F0822B83230E9477037B
:103BC0000E94FE0660E0C7010E941E0CEBCA832B18
:103BD000822BF4CF822B9091CB058927EFCFB114A4
:103BE00051F110FFEDCF402F429546954770440F9D
:103BF000440F802F8F70042E01C0880F0A94EAF7BB
:103C0000202F207104FF07C02FE030E001C0220FF9
:103C10004A95EAF72095169516951370123089F09B
:103C2000133069F03091CC05113041F0822B8323A1
:103C30000E947A03C5CF823018F2D5CF832B822B16
:103C4000F7CF822B9091CC058927F2CF1F70B1144A
:103C500039F0812F0E947D03802F0E944610B0CF43
:103C6000802F0E944F10812F0E948703A9CF023F0F
:103C700071F170F4003FC9F0013F91F0B11409F403
:103C800065C0A11409F45FC0802F0E94CF1198CFA6
:103C9000033F21F1043F91F78091CE0582FD2AC0B8
:103CA000812F8F71B11401F316C0B11469F0F5E0E2
:103CB000AF1608F085CF1F7181E090E0012E01C0A2
:103CC000880F0A94EAF7BECF26E0A216F2CF812F22
:103CD0008F71B110C9CF0E947D0372CF80E0B11403
:103CE00009F4A6CF1F7181E0012E01C0880F0A944C
:103CF000EAF79ECFB114C1F0809117058770843028
:103D000049F4109217051092190510921805812F89
:103D10008F71AACF35E063E0A31608F051CF812F51
:103D20008F710E94AC104CCF45E0A41640F0109269
:103D30001705109219051092180564E0F0CF81E084
:103D40000E9404043DCF812F8F71C5CFA114F9F2D9
:103D5000093349F45FEF83EF91E051508040904088
:103D6000E1F700C00000802F0E94361229CF0631F3
:103D7000BCE71B0709F01CCD809114058A7A91E0FD
:103D8000811101C090E09093120565E3811101C09B
:103D900069E286EB91E00E947007E4CB0631ECE724
:103DA0001E0709F005CD80911205811509F4FECC9E
:103DB00085E30E948A07D6CBA0E0B0E0E2EEFEE108
:103DC0000C9487318091E503803108F049C08091DF
:103DD000E403811509F444C0C091960389E0D82E0C
:103DE000809195038C17E1F1EC2EF12CDC9EE00123
:103DF0001124FE01E956FC4F84818115B1F19181B6
:103E00008091E003981331C090818091DF03981373
:103E10002CC08581811129C0028113818091E10329
:103E20009091E203081B190B60E08FED93E00E9474
:103E30001E0C0E94F30D08171907B8F48091E503D2
:103E40008F7080618093E503C356DC4F88818F704B
:103E5000806188838FED93E00E94E3160E94FA034D
:103E6000CDB7DEB7E7E00C94A331E7012196C77028
:103E7000B7CFAFE0B0E0EFE3FFE10C947F318C010E
:103E800086E0F801DE011A9601900D928A95E1F71D
:103E9000F801F580E4808FED882E83E0982E8091E4
:103EA000E303811117C0E11491F0F11409F480C10A
:103EB000C8010E944C0C811509F47AC189E0F8010F
:103EC000AFEDB3E001900D928A95E1F775DFFF2425
:103ED000F3946AC0A280B380D090E4038091E103A0
:103EE0009091E2033501681A790AD11409F411C1DD
:103EF000C080518060E08FED93E00E941E0C0E9414
:103F0000F30D6816790608F0B6C0E11401F380914C
:103F1000E003F8019181E090E503F0E1EF1608F08D
:103F200064C0981320C09091DF03F801808198133A
:103F30001AC02091E6033091E70387819085281706
:103F4000390789F4F1104BC08E2D8F7080618093FA
:103F5000E5038FED93E00E94E3168091E503F801FD
:103F60008683F12C21C0F1103AC040E0652D8C2DE4
:103F70000E94850940E0652D8C2D0E948509F82E50
:103F80008111EFCF8A859B850E94400C292F2295B5
:103F90002F70903470F49F702230A0F09115B1F022
:103FA000F8019681903190F48F2D2F96EFE00C94CC
:103FB0009B312A5F2F70223068F0C8010E94E316FF
:103FC000FD2CF2CF911511F0811571F3805E8830D0
:103FD00058F3F3CF803F40F3815F8330F9CF809176
:103FE000E50381608093E503BCCF98131EC09091D8
:103FF000DF03F8018081981318C02091E603309107
:10400000E703878190852817390779F4F1100DC0EF
:10401000E682C8010E94E31689E0F801AFEDB3E043
:1040200001900D928A95E1F752CFC8010E944C0C85
:10403000811509F4BDC0F11409F4BAC08091E503FB
:10404000803208F43BCF8091DF039091E0039A83A4
:104050008983BC82AB828091E3038D831E82EF82D1
:104060008091E6039091E70399878887CE010196B6
:104070000E94E31623CFD090E503F0E1DF1650F461
:104080008FED93E00E94E31689E0F40111928A9586
:10409000E9F767CFE11409F41ACF9091E003F80132
:1040A000818198131AC09091DF038081981315C005
:1040B0002091E6033091E70387819085281739071F
:1040C00061F4F1100AC0D682C8010E94E31689E0AB
:1040D000F40111928A95E9F7FACEC8010E944C0CBE
:1040E000811509F465C0F11409F462C08091E503FB
:1040F000803208F4E3CE8091DF039091E0039A834D
:104100008983BC82AB828091E3038D831E82DF8230
:10411000A7CF60E08FED93E00E941E0C0E94F30D8C
:104120006816790608F0B0CFE11409F4D0CEF11486
:1041300009F43EC09091E003F801818198132EC0EC
:104140009091DF038081981329C02091E60330917C
:10415000E703878190852817390701F58091E103EE
:104160009091E203A81AB90AF8ECAF16B10408F06E
:1041700053CF8091E50380FD4FCF803108F44CCFC1
:10418000F8018683982F907F903F09F442CF982FB3
:10419000907F905F8F70892B86833BCFC8010E94F0
:1041A0004C0C81118BCE8091E50381608093E503F7
:1041B000C8010E94E3168BCEA2E1B0E0E2EEF0E28D
:1041C0000C948A310A871B872C873D874E875F872F
:1041D000688B798B8A8BCE010A964BDE811128C0C1
:1041E000209195033091960389E0FE013A96DE0115
:1041F000119601900D928A95E1F78E858115C1F097
:10420000822F90E001968770992738171906D9F008
:1042100099E0929FD0011124A956BC4FFE0131961E
:1042200001900D929A95E1F7809395030E94FA030D
:1042300019E08091960390919503891312C06296BC
:10424000E4E00C94A6310E947D1310929503109225
:10425000960389E0EFEDF3E0DF011D928A95E9F71F
:10426000E7CF189FC001112489569C4F02DE8115AB
:1042700031F38091960390E001968770992780939F
:104280009603D7CFEF92FF920F931F93CF93DF93B5
:104290008091C805E091DE01CDE0811130C0CDB73D
:1042A000DEB7E6E00C94A431D1E0DE0FD093DE015E
:1042B000EE2EF12CCE9FF0011124E05AFA4F8481AA
:1042C0008115E1F087819085892B21F48185928584
:1042D000019651F4008111812281338144815581FD
:1042E00066817781808568DFCE9DF001CF9DF00DDE
:1042F0001124E05AFA4F148210921605ED2F809186
:10430000C805E81788F21092C8051092DE01C7CFE1
:10431000A4E0B0E0EEE8F1E20C947D3120915F057D
:10432000298397E0992E01E010E02DE0322E34E051
:10433000532E8824839480915E059981891307C048
:10434000A1DF0E9448062496E1E10C9499319981FD
:10435000892F90E09C838B83FC01EE0FFF1FEC5AAA
:10436000FA4F80819181989ED001999EB00D1124C1
:10437000FD01E45EFA4FFA83E983248121115BC0D9
:104380006090C805E0E6F5E060E070E0712C66152D
:1043900008F04FC0A384B484A981BA81CD90DC9089
:1043A0002FEF3FEF412C442D50E07601E40CF11C3F
:1043B000E40CF11CD701ED90FC90E114F10439F00C
:1043C000AE14BF0409F0A90143949A01ECCF2F3F2A
:1043D0003207D1F1D80102C0AA0FBB1F2A95E2F71C
:1043E0007A2A9801042C02C0220F331F0A94E2F7A4
:1043F000A901415051097416150629F5369EF001A0
:10440000379EF00D1124E05AFA4F989ED001999EE4
:10441000B00D1124A45EBA4F12962D913C911397C2
:104420003087278354821082118292878187159664
:104430008C920E9459068B819C8101969A83898374
:104440008370898378CF14826F5F7F4F3D969FCFB3
:104450001092CA051092C9051092110180915E0553
:1044600080935F050E9448060DCFACE1B0E0EBE31E
:10447000F2E20C947C314B8B5C8B6D8B7E8B8F8B43
:10448000B92E988FA92E911110921605188A198AA3
:104490001A8A86E0FE017396DE011A9601900D924B
:1044A0008A95E1F75F888091CE0582FF1FC00E9448
:1044B000E40F2091180530911905821B930B883861
:1044C000934138F08091170582FD03C082E00E947D
:1044D00004040E94E40F20911A0530911B05821BF1
:1044E000930B8838934110F00E9427045114D9F09F
:1044F0005E86BF8661E0CE010A960E941E0C61E0D6
:10450000CE010A960E941E0C61E0CE010A960E941E
:104510001E0C4C0180356CE7960791F4A11419F13B
:1045200081E0809311015E86BF860A851B852C85FC
:104530003D85452D5B2D688979898A893DDECDC011
:1045400081359C4721F4A11471F082DFECCF82E524
:1045500088168CE7980639F4A11429F0809111018E
:104560008111F3CFDDCF4CE1E42E45E0F42E412C58
:10457000612C712CD7016D917C91CC24CA94DD24DF
:10458000DA9480E0282F30E0FB01E80FF11DE80FFE
:10459000F11D408151814115510539F08416950670
:1045A00009F096018F5F6901EDCF10E0BFEFCB16E8
:1045B000DB0609F44EC0F70144811091110141114D
:1045C00010E0D70115963C90159716969C9116977A
:1045D000A11409F405C1111509F402C1311017C065
:1045E00021E030E00C2C01C0220F0A94EAF7922B54
:1045F00016969C9320915C0530915D052233310520
:1046000030F422E330E030935D0520935C05E1E077
:10461000F0E002C0EE0FFF1F8A95E2F7CF0101978D
:10462000D70116962C912817190699F4C090C90540
:10463000D090CA05C114D10409F453C00E94E40FFC
:104640008C199D09C39708F44CC081E0F70184835D
:1046500011E0412ABFEF6B1A7B0AE7E0EE0EF11C76
:10466000F8E06F16710409F085CFA11409F417C1A1
:10467000411409F414C10E94E40F9093CA05809379
:10468000C9058091C805883040F591E0980F909356
:10469000C80599E0FE013A96DE01119601900D924F
:1046A0009A95E1F75D82BE822DE0829FC0011124C0
:1046B000805A9A4F29E0FE013196DC0101900D925B
:1046C0002A95E1F72FEF3FEFDC011A963C932E93EA
:1046D00019971C969C928E921B976C96E2E10C9413
:1046E000983120915F0580915E05922FE0E0F0E027
:1046F00001E0281709F448C0422F50E0FA01EE0FFC
:10470000FF1FEC5AFA4F2080318037E0329DF001D4
:10471000339DF00D1124E45EFA4F608171817C8F2E
:104720006B8FB0E030E0A0E0EB8DFC8DEA0FF11D67
:10473000EA0FF11DC080D180C114D104E1F0F7016E
:104740000190F081E02DFA8FE98F30E007C0E1E0C1
:10475000C616D70609F0E0E0BE2B3F5FE98DFA8D63
:10476000E30FF11DE30FF11D60817181611571058A
:1047700071F7AF5FD9CFB11581F13A17C8F4E1E015
:10478000D7011496EC93F70190935F05EE15FF05A2
:1047900009F45FCF90E0FC01EE0FFF1FEC5AFA4FD7
:1047A0007182608201968370992780935E0551CF54
:1047B00037E0329DF001339DF00D1124E45EFA4F95
:1047C0000483EE15FF05F9F2291302C09F5F937071
:1047D0009A012F5F3F4F23708CCFE0E0F0E0F8CFDD
:1047E000292F30E0311024C061E070E002C0660F74
:1047F000771F8A95E2F7CB0101972817390791F0C7
:1048000010E0E1E0F0E002C0EE0FFF1FCA94E2F713
:104810006F01C094D70116968C9116978C2116962D
:104820008C9317CF411569F3C3010E945906E8CF55
:10483000A9010C2C02C0559547950A94E2F7C901CD
:10484000019782239323892B39F540FF25C0D70197
:1048500012968D919C91892BD1F087E0FE013196C3
:10486000DF011D928A95E9F70E94E40F9C018B837A
:104870009C8384E08D83F70192818381792F9887CF
:10488000898709811A8144E05E816F8195DCD701B7
:1048900015961C92132DB5CF142F1170B2CF909195
:1048A0005F0580915E05981731F032DDB1E04B165F
:1048B00009F413CF38CEE6DC1092CA051092C90570
:1048C0000E944806F3CFA6E0B0E0E9E6F4E20C94DB
:1048D0008A310E94E40F8C018091890390918A03B0
:1048E0008017910771F019821A820E94E40FBC01AF
:1048F00049815A8180E090E0B8DD10938A030093EB
:1049000089032696E4E00C94A631A6E0B0E0EBE83B
:10491000F4E20C948C319093860380938503811587
:1049200020E2920730F40E9421122696E2E00C94D5
:10493000A83180EF89838A830E94E40F8160BC01E3
:1049400049815A8181E091E090DDEFCFA6E0B0E0AF
:10495000ECEAF4E20C948A318C0190938603809304
:104960008503011580E21807B0F4802F0E943612EB
:10497000C801805E9109089728F06EE570E1011585
:10498000110511F46FE470E1C8010E946E032696D0
:10499000E4E00C94A63180EF89838A830E94E40FBF
:1049A0008160BC0149815A8181E090E05EDDEFCFFA
:1049B000CF93DF93D82FC92FA8DF8D2F9C2FC6DF71
:1049C000DF91CF9108950F931F93CF93DF938C01C5
:1049D000862F6EEF73E00E94DE0D892B91F4C0915B
:1049E000FE03D091FF03209761F0F80182818330AC
:1049F00039F4CE01DDDFCE01DBDFCE01D9DF01C02E
:104A0000E0F7DF91CF911F910F9108950F931F93BE
:104A1000CF93DF938C01EB016EEF73E08C2F0E943C
:104A2000DE0D892B09F057C0FE01FF27D801129631
:104A30008C911297E05DFD4F8130A9F415968C9111
:104A400082FD4EC080FF4CC082E0808380910004D4
:104A5000909101040097B9F48091FE039091FF03B7
:104A60000097C9F110C08230A1F515968C9182FD96
:104A700026C080FD0AC083E080838091020490916B
:104A800003040097F1F041DF26C084E08083809129
:104A90000404909105040097B1F78091FE03909172
:104AA000FF03009701F184DF8091000490910104DD
:104AB000009749F78091FE039091FF03E4CF85E0D2
:104AC00080838091FE039091FF03009721F070DFB7
:104AD000F1CF86E08083DF91CF911F910F910895F0
:104AE00081E08083B9CF8091000490910104B8CF18
:104AF0000F931F93CF93DF938C01EB016EEF73E065
:104B00008C2F0E94DE0D892B71F4DD27C05DDD4FF7
:104B10008881F801128218828330E9F048F48130EC
:104B200059F0823081F0DF91CF911F910F9108955C
:104B30008430B1F08530B9F78091FE039091FF0386
:104B4000009789F306C080910004909101040097BA
:104B500099F3FCDEE8CF8091020490910304F7CF33
:104B60008091040490910504009799F72091FE0329
:104B70003091FF03809100049091010421153105CB
:104B8000F9F2009731F7C901E4CFCF93DF93A9E39E
:104B9000B1E06EE371E041E030E02D912F3F79F01C
:104BA000E22FE295EF70E05EF0E0808190E02F7000
:104BB00002C0959587952A95E2F780FF22C080E094
:104BC000382B440F6A177B0741F780914902831302
:104BD0001AC08091C001811509F1C091BE01D09128
:104BE000BF010E94E40F8C1B9D0B0597B8F08091CC
:104BF0004902909181038913809381031092C0012F
:104C00000DC0842FDDCF3093490281E08093C00135
:104C10000E94E40F9093BF018093BE01DF91CF917A
:104C20000895CDB7DEB7E0970FB6F894DEBF0FBE9C
:104C3000CDBF85B7806885BF85B7806885BF84B7DD
:104C4000877F84BF0FB6F894A89580916000886133
:104C500080936000109260000FBE80E890E00FB675
:104C6000F89480936100909361000FBE81E080937F
:104C7000030181E296E09093B5018093B4010E9414
:104C800030060E941D0D0E94600D8BE0E5E1F1E011
:104C9000DE01119601900D928A95E1F7FE013196A1
:104CA0009E01245F3F4FEFA7F8AB41E050E08191B8
:104CB000A82FA295AF70B0E091966C9191978F70EC
:104CC0008A0102C0000F111F8A95E2F7C801962FD2
:104CD000982B91969C93919792969C919297809500
:104CE000892392968C93E217F30709F7879A8091AC
:104CF0004C0280FFE9C08F9A0E94CE080E942B09C7
:104D00008091E20084608093E20078948091840333
:104D1000811599F08091E9001091EC008F70179542
:104D200011271795182B1092E9008091E80083FD58
:104D30000E94B7131F701093E90082E084BD93E0D6
:104D400095BD9DE797BD80936E000E948E0C8111EA
:104D500002C00E94490EEFE6F3E088E0DF011D92F9
:104D60008A95E9F78098889884988C9810926403C3
:104D700010926203109263038FEF93E09093DB0233
:104D80008093DA021092D9021092D8021092D702C0
:104D90001092D602109259021092580210925702A5
:104DA0001092560210926C0310926B039093610361
:104DB0008093600310925F0310925E0310925D0374
:104DC00010925C031092DF021092DE021092DD025C
:104DD0001092DC0210926A03109269031092680329
:104DE000109267031092660310926503A9E3B1E085
:104DF0002EE331E041E050E08D918F3FA1F0E82FAC
:104E0000E295EF70F0E061A18F708A0102C0000F9F
:104E1000111F8A95E2F7C801902F9095962391A3D0
:104E200092A1892B82A32A173B0731F710928103A5
:104E30001092490280E090E00E942132833E9E4F12
:104E400021F40E948E0C81111DC063EE7EEF80E084
:104E500090E00E944F3260E082E090E00E943532A4
:104E600081E08093CB0561E083E090E00E943532E1
:104E700060E074E184E090E00E944F320E94490EAD
:104E80000E94A40982E090E00E94143280934C02B8
:104E900084E090E00E9421329093CE058093CD056E
:104EA00074DE8FE59AEE0197F1F700C000006DDE29
:104EB0008091810383FF0AC06FEF7FEF80E090E075
:104EC0000E944F320E9413088F9816CF83E090E023
:104ED0000E9414320E9477030E94E10E8FE090E05E
:104EE0000E941C326093CF057093D0058093D1054A
:104EF0009093D205663010F00E94A409E091CF058E
:104F0000F0E0EE0FFF1FE655FE4F808191810E9479
:104F1000D10E84E091E090938C0380938B0382E028
:104F2000282E3324339480918403853049F4809172
:104F30008403853009F434C10E947D130E94FE066B
:104F400024DE80914D02E09081038E11C6C6BBDC49
:104F500000918504109186040115110591F1C0900E
:104F60005202D0905302E0905402F09055020E94F9
:104F7000C6076C197D098E099F09C0904E02D0901A
:104F80004F02E0905002F09051026C157D058E05A5
:104F90009F05B8F0C8010E94211210928604109259
:104FA00085041092520210925302109254021092F1
:104FB000550210924E0210924F021092500210921F
:104FC0005102E0900D05F0900E05E114F10441F15D
:104FD00000910F05109110050E94E40F9C01201B09
:104FE000310B8901C7010E94F30D80179107C0F4AE
:104FF00020910D0530910E05C9019927287F33278F
:10500000232B09F019C114E0880F991F1A95E1F7B5
:1050100083579B4FDC0115962C9122FF0E94841030
:1050200080911101811511F10091C9051091CA05F6
:1050300001151105D9F00E94E40F801B910B2091FE
:105040005C0530915D052817390780F490915F0564
:1050500080915E05981709F4F2C05AD910925D0547
:1050600010925C051092CA051092C90580917703D1
:10507000811551F010927703809171038093720330
:1050800080916F038093700380EFF8D72C0184EF39
:10509000F5D73C0180916C03811521F080916B0361
:1050A00081112BC0EBE6F3E0FF93EF932CE633E0A6
:1050B0003F932F93E6E58E2EE2E09E2EF8E5AF2E8D
:1050C000F2E0BF2EAAE5CA2EA2E0DA2EB8E9EB2E56
:1050D000B2E0FB2E06ED12E027ED32E048ED52E0A3
:1050E0006AED72E0C2010E943C02909368038093D3
:1050F00067030F900F900F900F9080916A038115B6
:1051000021F08091690381112BC069E673E07F93E0
:105110006F93AAE6B3E0BF93AF934CED842E42E0C9
:10512000942E5EEDA52E52E0B52E60EEC62E62E006
:10513000D62E7EE1E72E73E0F72E0CE513E02DE589
:1051400033E04EE553E060E673E0C3010E943C02A9
:1051500090936603809365030F900F900F900F90CC
:1051600040916703509168038091650390916603B5
:1051700020916403211178C04416550608F067C0D9
:105180006816790608F480C083E0809364038091F8
:105190006303811509F478C01092630311E075C0B0
:1051A00080918403843031F10E94790A10924A027E
:1051B000A8E1B0E0E0E40FB6F894A895A0936000F1
:1051C0000FBEE093600083B7817F846083BF83B7A5
:1051D000816083BF7894889583B78E7F83BF0FB635
:1051E000F894A89580916000886180936000109287
:1051F00060000FBECADC80918103811509F497CE4F
:1052000080914B02811509F492CE19BCF2E0F9BDF0
:1052100009B400FEFDCF8091D8008F7D8093D80027
:105220008091E00082608093E0008091E00081FD49
:10523000FCCF0E947D137BCE80E090E0EBCE22D8A5
:105240001092CA051092C9050E9448060FCF681631
:105250007906D0F430926403809162038115A1F045
:10526000109262031FEF11C0213009F079C044167B
:10527000550608F46EC06816790630F01092640383
:10528000209363031092620310E0E090FC03F0901F
:10529000FD030E94E40F8E199F0984369105B0F139
:1052A000E0906D03F0906E030E94E40F8E199F0949
:1052B000059760F18091FB03811128C0111531F130
:1052C0008091710390E09C012F5F3F4F2370332743
:1052D000409172034217130699F081599C4F41E0A7
:1052E000113009F040E0479544274795DC011496BA
:1052F0004C932093710380916F038F5F80936F03B2
:105300000E94E40F90936E0380936D0380E01AED8A
:105310002091720390917103921709F458C030E004
:10532000F901ED58FC4F808187FB882780F92F5FBA
:105330003F4F2370332720937203909170039F5F38
:1053400090937003B12FB81B8B2F0E947A1281E0CB
:10535000DFCF6816790608F097CF2092640390CFCC
:10536000223001F54416550670F06816790608F0EB
:105370008BCF3092640380916203811509F484CF4E
:10538000109262030BCF6816790608F47DCF83E094
:105390008093640380916303811509F475CF1092A3
:1053A000630360CF4416550658F06816790608F472
:1053B0006BCF10926403309262031092630364CF48
:1053C0006816790608F060CF20926403F4CF81114B
:1053D0000E94C6070E94790A81110E94C60786E0D2
:1053E000EEEEF3E0AFA5B8A901900D928A95E1F732
:1053F0001092F0031092F1031092F2031092F30353
:105400008B819C81892B811509F443C000917A031B
:1054100010917B030E94E40F9C01201B310B9091A3
:10542000EC03911509F454C42531310590F19F3FE7
:1054300019F09F5F9093EC031B81111559F00E94A6
:10544000B40691E011160CF09FEF899F802D112476
:105450008093F0031C81111559F00E94B40691E06D
:1054600011160CF09FEF899F802D11248093F1037A
:105470008091F003811569F01091F103111549F045
:105480000E94A6068093F003812F0E94A6068093B7
:10549000F1038D819E81892B811509F443C0009110
:1054A0007803109179030E94E40F9C01201B310BBB
:1054B0009091EB03911509F406C42135310590F163
:1054C0009F3F19F09F5F9093EB031D81111559F0D9
:1054D0000E94D40691E011160CF09FEF899F802D59
:1054E00011248093F2031E81111559F00E94D406F5
:1054F00091E011160CF09FEF899F802D112480936D
:10550000F3038091F203811569F01091F3031115F3
:1055100049F00E94A6068093F203812F0E94A606FE
:105520008093F3036FA578A98EEE93E00E9496070F
:1055300081110CC08091F0039091F103892B90911F
:10554000F203892B9091F303892B81110E94D710CC
:1055500086E0EFA5F8A9AEEEB3E001900D928A9532
:10556000E1F70E94FE0690917C03891721F0809359
:105570007C030E94C60780918403843009F0D3CC59
:1055800083E08093E9008091E80082FFCCCC809199
:10559000E80090E085FF05C00E949D08811519F183
:1055A00091E08091E8008B778093E800911509F4F1
:1055B000BACC0091870310918803E9810115110588
:1055C00071F1EE3F09F04DC08A81833020F08550A3
:1055D000833008F046C0EA81EE3008F042C0F0E0C7
:1055E000EB5BFB4CE7C600E210E0FE0131967F0169
:1055F0008091E80085FD0AC08091E8008B77809358
:10560000E8000E949D08811599F3CACF8091F100AE
:10561000D7018D937D010150104051F7C1CFE43186
:1056200048F4E11549F0E150E33130F4F0E0ED5A8F
:10563000FB4CC0C6EE3F79F28FEF898312C01A820D
:1056400089E08B830EC08A81823081F08330B1F093
:10565000813091F70E94C607B3D66B837C838D831C
:105660009E83CE0101960E94ED085DCC88E290E019
:10567000DBD61B821C821D828E83F3CF8091820336
:1056800090918303892B69F380918103DACF8A811A
:10569000823091F66B817C818D819E8191D688E2EA
:1056A00090E0E3D6DECF4C816B818A810E94B00B03
:1056B0009827892798279E838D83D3CF2D813E817C
:1056C0003227232732274C816B818A810E94320A3C
:1056D000C8CF0E94A70CC5CF80E18A83C2CF82E0E9
:1056E0008A838FEAAECF8C818D3108F0BACF8A8061
:1056F0009B80982489249824A12CB12C8E010F5FC3
:105700001F4F7801E80EF11C0E151F0509F4A9CFF3
:1057100080E0BFEA8B16B2E09B06A104B10420F43E
:10572000C4018F5A9E4F80D6F80184830F5F1F4FAC
:10573000FFEF8F1A9F0AAF0ABF0AE6CF809182035C
:1057400090918303892B09F48CCF8C818D3108F0E3
:1057500088CF882E912CA12CB12CCA80DB80DC2430
:10576000CD24DC24E12CF12C8E010F5F1F4F412C46
:10577000512C3201481459046A047B0408F071CF9B
:105780002FEAC21622E0D206E104F10438F4D8016F
:1057900014966C91C6018F5A9E4F67D6BFEF4B1A75
:1057A0005B0A6B0A7B0AEFEFCE1ADE0AEE0AFE0AEC
:1057B0000F5F1F4FDFCF0E940E0E53CF84E08DCFBF
:1057C0008C818D3108F04DCF882E912CA12CB12CDD
:1057D000CA80DB80DC24CD24DC24E12CF12C412C9C
:1057E000512C32018E010B5F1F4F481459046A047B
:1057F0007B0408F036CF80E0F8E2CF16D104E10454
:10580000F10418F4C60189960FD6D8018D938D0145
:10581000BFEF4B1A5B0A6B0A7B0AEFEFCE1ADE0A68
:10582000EE0AFE0AE2CF2C81622E712C2D3108F097
:1058300018CF8A819B819827892798274C01A12C12
:10584000B12C8832910508F00CCF422F50E060E077
:1058500070E04BA75CA76DA77EA748E250E060E030
:1058600070E0481959096A097B0942175105610519
:10587000710508F4F6CE2091820330918303232B27
:1058800009F03EC07C0159E2E50EF11C80FBCC24FE
:10589000DD24C0F880FF0BC08896C6D59D8189277E
:1058A0009827892781159C4711F48FEF8D838BA54D
:1058B0009CA5ADA5BEA5880D991DAA1DBB1D80FF89
:1058C00017C083010150110935E0432E512C4C0EB5
:1058D0005D1E400E511EC701860D971DA5D5D20134
:1058E0009C9181159C4719F48FEFF2018083380158
:1058F000FE013196EC0DFD1D2FEFC614D70438F0D4
:105900008E010F5F1F4FC12CD12C760124C09481D2
:10591000858181159C4711F42483258312E0C10EF3
:10592000D11C3296EACF28E282169104A104B10478
:1059300030F4D80114966C91C401899696D5BFEFC6
:10594000CB1ADB0AEB0AFB0AEFEF8E1A9E0AAE0AAD
:10595000BE0A0F5F1F4F2BA53CA54DA55EA5C21625
:10596000D306E406F506F8F27CCE8091820390918E
:105970008303892B09F475CECE0101960E94ED08B0
:105980003FEF40E752E0315040405040E1F700C067
:10599000000098CA88E0E1E2F1E0DE019196019012
:1059A0000D928A95E1F7FE0132968FE1DF011D929B
:1059B0008A95E9F786E0898388E07F96DE0115966F
:1059C00001900D928A95E1F74CCE80E3898381E0C6
:1059D0008A831B821C8245CE8B819C81092E000C00
:1059E000AA0BBB0B25E0880F991FAA1FBB1F2A9586
:1059F000D1F7AC01BD01405E5F4F6F4F7F4F48173D
:105A000059076A077B0708F42CCE8033E1E09E0734
:105A1000A105B10508F025CE4133F1E05F0761052E
:105A2000710520F040E351E060E070E0481B590B45
:105A3000BC01645F7C4FCE010196C9D412CE4AE10D
:105A400050E06FEF70E0CE010796D7D480918203CB
:105A500089830A831B8283E08C831D8285E00CCEC0
:105A600081E090E0909388038093870382E390E045
:105A70009093800380937F030E94E40F90937E03B2
:105A800080937D03EECD0115110571F1D090810356
:105A9000E0907D03F0907E030E94E40F8E199F0931
:105AA0008536910540F1D5FE26C0D3FE24C00E9464
:105AB000E40F90937E0380937D0380917F03909108
:105AC000800301979093800380937F03892B61F477
:105AD000109288031092870381E090E090938303F3
:105AE0008093820300E010E08091820389830A831F
:105AF00080917F03A6CD82E390E090938003809312
:105B00007F03F2CF1092830310928203AACD40E26A
:105B100050E06FEF70E0CE0101966FD4A2CDEB8123
:105B2000E73008F09ECDF0E0EA59FB4C43C4FE019B
:105B300034968DE1DF011D928A95E9F788E089832B
:105B40008A837FCD8C819AE0F92E8E010F5D1F4FE5
:105B5000F8012F2D11922A95E9F7B8010E94DE0D68
:105B60008983F801DE01129601900D92FA94E1F713
:105B700078CD1C818AE0FE013596DE019196019078
:105B80000D928A95E1F789A19AA10E9423069AA312
:105B900089A38BA19CA10E9423069CA38BA38DA10A
:105BA0009EA10E9423069EA38DA38FA198A50E946B
:105BB000230698A78FA38FEF183060F43AE0139F65
:105BC000B00111246F597F4F4AE050E0CE01819619
:105BD0006AD480E089830E94300643CD2C816AE03C
:105BE000CE018196DC01E62F1D92EA95E9F7283077
:105BF00008F044C0629FB00111246F547F4F4AE007
:105C000050E002D480E089838AE0FE01B196DE0193
:105C10001296D6CE1C818AE0FE013596DE01919661
:105C200001900D928A95E1F789A59AA50E94230615
:105C30009AA789A78FEF183060F4FAE01F9FB00190
:105C400011246F547F4F4AE050E0CE0181962BD44F
:105C500080E089830E941D0D04CD2C816AE0CE0175
:105C60008196DC01E62F1D92EA95E9F7283030F4A1
:105C7000629FB00111246F5F7E4FC1CF8FEFC3CF02
:105C80001C818AE0FE013596DE01919601900D920D
:105C90008A95E1F78BA19CA10E9423069CA38BA36C
:105CA0008FEF183060F4FAE01F9FB00111246F5F8E
:105CB0007E4F4AE050E0CE018196F5D380E08983A3
:105CC0000E94600DCECC2B30310508F0FBCB2ACCE6
:105CD0002B30310508F0ADCBDCCBF82EFE2400E0F4
:105CE00011E08F2D81238115A9F009831A820E946A
:105CF000E40F9C838B833D8291E08E2D8123811163
:105D000001C090E09E8349815A816B817C818D81A5
:105D10000E9435220F5F110F053019F7E0924D02F6
:105D20000E94C60715C978941F921FB61F921124AE
:105D30008F939F93AF93BF938091D6019091D7019A
:105D4000A091D801B091D9010196A11DB11D8093F8
:105D5000D6019093D701A093D801B093D901BF91F8
:105D6000AF919F918F911F901FBE1F9018951F920A
:105D70000F920FB60F9211242F933F934F935F937F
:105D80006F937F938F939F93AF93BF93EF93FF9303
:105D90008091E10082FF09C08091E20082FF05C08E
:105DA0008091E1008B7F8093E1008091DA0080FF99
:105DB00023C08091D80080FF1FC08091DA008E7FC1
:105DC0008093DA008091D90019BC80FFA6C082E0E0
:105DD00089BD09B400FEFDCF81E0809384038091EA
:105DE000C501811109C00E94CE080E942B09809133
:105DF000E20084608093E2008091E10080FF1AC09D
:105E00008091E20080FF16C08091E2008E7F809337
:105E1000E2008091E20080618093E2008091D800EE
:105E200080628093D80019BC85E08093840383E06E
:105E3000809303018091E10084FF2EC08091E200F5
:105E400084FF2AC019BC82E089BD09B400FEFDCFE1
:105E50008091D8008F7D8093D8008091E1008F7E63
:105E60008093E1008091E2008F7E8093E200809138
:105E7000E20081608093E2008091C401811509F401
:105E800051C084E08093840380918403843009F0BE
:105E900051C082E0809303018091E10083FF2CC018
:105EA0008091E20083FF28C08091E100877F80938A
:105EB000E10082E0809384031092C4018091E100AC
:105EC0008E7F8093E1008091E2008E7F8093E200DC
:105ED0008091E20080618093E20042E060E080E037
:105EE0000E94FB088091F00088608093F00081E0C0
:105EF0008093030180930201FF91EF91BF91AF91D5
:105F00009F918F917F916F915F914F913F912F91D1
:105F10000F900FBE0F901F9018951092840310924F
:105F2000C5016ACF8091E30087FF02C083E0AACF5A
:105F300081E0A8CF81E0AECF1F920F920FB60F92F3
:105F40001124EF92FF920F931F932F933F934F9340
:105F50005F936F937F938F939F93AF93BF93CF93F1
:105F6000EF93FF9309EE10E0F8018081C091EC00FF
:105F70008F70C795CC27C795C82B108280EFE82E6D
:105F8000F12CF7018081877F808378940E94B7137A
:105F9000F8011082F701808188608083CF70F8015A
:105FA000C083FF91EF91CF91BF91AF919F918F915E
:105FB0007F916F915F914F913F912F911F910F9121
:105FC000FF90EF900F900FBE0F901F901895803F9D
:105FD00009F188F4843901F140F48533F9F086330E
:105FE000F9F0843339F583E208958639D9F0873999
:105FF00009F582E20895853FB9F030F4813FB1F0B0
:10600000843FC1F484E00895863F91F0873F91F486
:1060100087E0089580E0089580E2089584E208957D
:1060200085E2089581E2089585E0089581E008956C
:1060300086E008958FE1089595E890937A00982F6F
:106040009072906890937B008F7190911201892BD0
:1060500080937C0080917A00806480937A008091A4
:106060007A0086FDFCCF8091780020917900909194
:106070007A009F7790937A00922F0895A8DFDCCF63
:10608000289A219A229A23982B9880E58CBD08950E
:10609000FC01809114018F3F09F085C080818F3F02
:1060A00009F481C01092D4058181811519F080E234
:1060B0008093D40592818091D405923009F44FC029
:1060C000933009F450C08460913009F449C0838151
:1060D000948121E030E02817390708F446C0809108
:1060E000D4052032310509F456C008F041C02830EB
:1060F000310509F44BC02031310509F44AC0223082
:10610000310509F43FC08CB59091D405892B8CBD25
:106110008091D305811519F08DB581608DBD2081E9
:1061200020931401458140931301E22FE295EF7013
:10613000A1E2AE0FB0E03C912F7081E090E001C091
:10614000880F2A95EAF7232F282B2C93EE5DF0E099
:106150009081411125C0892B808381E0089588605A
:106160008093D405B4CF8C60FBCF220F331FB3CF05
:106170002034310599F083602038310521F6809371
:10618000D405C1CF81E08093D305BDCF91E090933A
:10619000D3058160F4CF91E09093D3058260EFCF77
:1061A00080958923D9CF80E00895A6E0B0E0EAED9C
:1061B000F0E3B2C089836A834B833D832C8381E003
:1061C0008E83CE01019664DF2696E2E0C1C0CF93B4
:1061D000DF938EBD0E94E40FEC010DB407FE05C0F5
:1061E0008EB590E0DF91CF9108950E94E40F8C1B53
:1061F0009D0B8436910588F38EEF9FEFF3CFCF93FD
:10620000DF931EBC0E94E40FEC010DB407FE05C035
:106210008EB590E0DF91CF9108950E94E40F8C1B22
:106220009D0B8436910588F38EEF9FEFF3CF0F938C
:106230001F93CF93DF93EC018C01060F171FC0173C
:10624000D10739F480E090E0DF91CF911F910F9159
:1062500008958991BCDF97FFF2CF8EEF9FEFF4CFC7
:106260000F931F93CF93DF93EC018C01060F171F41
:10627000C017D10739F480E090E0DF91CF911F91F2
:106280000F910895BCDF97FD02C08993F1CF8EEF87
:106290009FEFF3CF209114012F3F51F1E22FE295B0
:1062A000EF70A1E2AE0FB0E03C912F7081E090E082
:1062B00001C0880F2A95EAF7232F282B2C93EE5D37
:1062C000F0E0209113019081211599F0892B8083B2
:1062D0008FEF809314018DB58E7F8DBD9CB580911D
:1062E000D405809589238CBD1092D4051092D305D6
:1062F000089580958923EBCF2F923F924F925F9222
:106300006F927F928F929F92AF92BF92CF92DF92C5
:10631000EF92FF920F931F93CF93DF93CDB7DEB72A
:10632000CA1BDB0B0FB6F894DEBF0FBECDBF0994BE
:106330002A88398848885F846E847D848C849B8415
:10634000AA84B984C884DF80EE80FD800C811B8123
:10635000AA81B981CE0FD11D0FB6F894DEBF0FBE52
:10636000CDBFED010895AA1BBB1B51E107C0AA1FB9
:10637000BB1FA617B70710F0A61BB70B881F991FE6
:106380005A95A9F780959095BC01CD01089597FB8A
:10639000072E16F4009406D077FD08D0E4DF07FC42
:1063A00005D03EF4909581959F4F08957095619525
:1063B0007F4F0895EE0FFF1F0590F491E02D099493
:1063C0006927962769277827872778270895FB016B
:1063D000DC0102C005900D9241505040D8F708955D
:1063E000FB01DC0104C08D910190801921F4415022
:1063F0005040C8F7881B990B0895DC0101C06D93CC
:1064000041505040E0F70895DC01CB01FC01F999BF
:10641000FECF06C0F2BDE1BDF89A319600B40D92F0
:1064200041505040B8F70895F999FECF92BD81BD13
:10643000F89A992780B50895A6E1B0E044E050E0CD
:10644000E5CFA8E1B0E042E050E0E0CFDC01A40FEE
:10645000B51F4150504040F0CB01840F951F2E9145
:1064600005D041505040D8F70895262FF999FECF16
:1064700092BD81BDF89A019700B4021639F01FBA97
:1064800020BD0FB6F894FA9AF99A0FBE08950396B4
:10649000272FECDFEADF252FE9DF242FE7CF019656
:1064A000272FE4DFE2CFDC01CB0102C02D9105D024
:1064B00041505040D8F70895262FF999FECF1FBAC2
:1064C00092BD81BD20BD0FB6F894FA9AF99A0FBE1D
:1064D000019608955058BB27AA270ED0E5C0D6D004
:1064E00030F0DBD020F031F49F3F11F41EF4CBC02C
:1064F0000EF4E095E7FBC1C0E92FE7D080F3BA17AF
:10650000620773078407950718F071F49EF5FFC0C2
:106510000EF4E0950B2EBA2FA02D0B01B9019001BE
:106520000C01CA01A0011124FF27591B99F0593F02
:1065300050F4503E68F11A16F040A22F232F342F4A
:106540004427585FF3CF469537952795A795F04098
:106550005395C9F77EF41F16BA0B620B730B840BAD
:10656000BAF09150A1F0FF0FBB1F661F771F881F65
:10657000C2F70EC0BA0F621F731F841F48F48795BD
:1065800077956795B795F7959E3F08F0B3CF9395AC
:10659000880F08F09927EE0F97958795089504D0F6
:1065A0006894B111B5C0089598D088F09F5790F0C5
:1065B000B92F9927B751A0F0D1F0660F771F881F28
:1065C000991F1AF0BA95C9F712C0B13081F09FD067
:1065D000B1E008959CC0672F782F8827B85F39F005
:1065E000B93FCCF3869577956795B395D9F73EF487
:1065F00090958095709561957F4F8F4F9F4F08952F
:10660000E89409C097FB3EF490958095709561954C
:106610007F4F8F4F9F4F9923A9F0F92F96E9BB2702
:106620009395F695879577956795B795F111F8CF7E
:10663000FAF4BB0F11F460FF1BC06F5F7F4F8F4FE9
:106640009F4F16C0882311F096E911C0772321F0DF
:106650009EE8872F762F05C0662371F096E8862F77
:1066600070E060E02AF09A95660F771F881FDAF7CE
:10667000880F9695879597F9089597F99F6780E811
:1066800070E060E008959FEF80EC089500240A9484
:106690001616170618060906089500240A941216FD
:1066A0001306140605060895092E0394000C11F430
:1066B000882352F0BB0F40F4BF2B11F460FF04C0DD
:1066C0006F5F7F4F8F4F9F4F089557FD9058440F36
:1066D000551F59F05F3F71F04795880F97FB991F41
:1066E00061F09F3F79F087950895121613061406FE
:1066F000551FF2CF4695F1DF08C01616170618068B
:10670000991FF1CF86957105610508940895E89465
:10671000BB2766277727CB0197F908950BD0C4CF05
:10672000B5DF28F0BADF18F0952309F0A6CFABCF7C
:106730001124EECFCADFA0F3959FD1F3950F50E05F
:10674000551F629FF001729FBB27F00DB11D639F23
:10675000AA27F00DB11DAA1F649F6627B00DA11DC9
:10676000661F829F2227B00DA11D621F739FB00D6F
:10677000A11D621F839FA00D611D221F749F3327DF
:10678000A00D611D231F849F600D211D822F762F78
:106790006A2F11249F5750408AF0E1F088234AF075
:1067A000EE0FFF1FBB1F661F771F881F91505040C1
:1067B000A9F79E3F510570F060CFAACF5F3FECF381
:1067C000983EDCF3869577956795B795F795E795AD
:1067D0009F5FC1F7FE2B880F911D9695879597F9BE
:1067E0000895F894FFCFFE10041107110D11221126
:1067F0002211221122112211221122112211101113
:10680000151119111F1144114A114E119814BE147B
:10681000C414BE14C41417153915C41440164D16EB
:10682000601BC81B681B331B371B6C1B3B1B701B7F
:106830007C1B471BC11B4B1B801B4F1B841BA91BB5
:10684000531B881BB01B581B8E1B961B3F1B741BB6
:10685000431B781B5C1B921BA01BB91BBF1B2D1B72
:10686000641BCF1B001B061BF31AFA1A0C1B121B0E
:10687000181BA81CA81CE11CE11C931DAE1D071DC4
:10688000071DB31D261E371E371ECA2CE52CEC2C07
:10689000312B312B1F2D302D432D822D872D312B68
:1068A000312B312B8F2D1F2B232B472B532B5E2B63
:1068B000692B1C2B1C2B1C2B1C2BB52C6C2B6F2B16
:1068C000732B9E2BDB2BDE2BE02B132C972DA22D75
:0A68D000B92DEE2D0A2E2D2E402EBC
:1068DA0000000100C307FC092408120A170AF30979
:1068EA0001014001FF91933436379667F6F5F3F7C5
:1068FA0000EE5B21B355DF2BA60044227B4901271A
:10690A0001AC004F02680288029492C63597E200F1
:10691A00E900EA00B500B600B700CD008301CC005B
:10692A008A019201940121022302240225022602ED
:10693A0027022A02B300B4006F0070009F01CB0146
:10694A009F02A002E200E900EA00B500B600B70023
:10695A00CD008301CC008A01920194012102230215
:10696A0024022502260227022A02B300B4006F007D
:10697A0070009F01CB019F02A00258028403B00459
:04698A00400660095A
:00000001FF
